:020000040000FA
:0408000098EF0BF072
:1008100003B275EF05F0F2B493EF05F09EB09BEFD5
:1008200005F09EB2A3EF05F0F2A81AEF04F0F2B2C1
:1008300023EF04F0F2B01FEF04F047EF0BF0F29655
:10084000F29047EF0BF0CD90F2929EA02DEF04F0C6
:100850000101533F2DEF04F0542BB2C1B6F1B3C1E7
:10086000B7F1B4C1B8F1B5C1B9F1AEC1B2F1AFC120
:10087000B3F1B0C1B4F1B1C1B5F1AAC1AEF1ABC130
:10088000AFF1ACC1B0F1ADC1B1F1A6C1AAF1A7C140
:10089000ABF1A8C1ACF1A9C1ADF1A2C1A6F1A3C150
:1008A000A7F1A4C1A8F1A5C1A9F19EC1A2F19FC160
:1008B000A3F1A0C1A4F1A1C1A5F19AC19EF19BC170
:1008C0009FF19CC1A0F19DC1A1F1CECF9AF1CFCFF4
:1008D0009BF153C19CF154C19DF1CF6ACE6A0101D5
:1008E000536B546B9E90CD800FBC0F8E0FBA7CEF74
:1008F00004F00F8A47EF0BF013880F8C0FBEB9EF8F
:1009000004F09AC19EF19BC19FF19CC1A0F19DC1D1
:10091000A1F19EC1A2F19FC1A3F1A0C1A4F1A1C107
:10092000A5F1A2C1A6F1A3C1A7F1A4C1A8F1A5C1D7
:10093000A9F1A6C1AAF1A7C1ABF1A8C1ACF1A9C1A7
:10094000ADF1AAC1AEF1ABC1AFF1ACC1B0F1ADC177
:10095000B1F1AEC1B2F1AFC1B3F1B0C1B4F1B1C147
:10096000B5F1B2C1B6F1B3C1B7F1B4C1B8F1B5C117
:10097000B9F101015E6B5F6B606B616B9A515E2731
:100980009B515F239C5160239D5161239E515E27A3
:100990009F515F23A0516023A1516123A2515E2783
:1009A000A3515F23A4516023A5516123A6515E2763
:1009B000A7515F23A8516023A9516123AA515E2743
:1009C000AB515F23AC516023AD516123AE515E2723
:1009D000AF515F23B0516023B1516123B2515E2703
:1009E000B3515F23B4516023B5516123B6515E27E3
:1009F000B7515F23B8516023B9516123D8900101E9
:100A0000613360335F335E33D8900101613360330B
:100A10005F335E33D8900101613360335F335E33FF
:100A200000C10CF101C10DF102C10EF103C10FF1C2
:100A300004C110F105C111F106C112F107C113F192
:100A400008C114F109C115F10AC116F10BC117F162
:100A500034C135F111B838EF05F00101620E046FB1
:100A6000010E056F000E066F000E076F41EF05F0D7
:100A70000101A70E046F020E056F000E066F000E37
:100A8000076F5EC100F15FC101F160C102F161C198
:100A900003F1B1EC30F003BF04D01CBE02D01CA0A7
:100AA000108C11A059EF05F010BA59EF05F00F8026
:100AB000108A0CC100F10DC101F10EC102F10FC18C
:100AC00003F110C104F111C105F112C106F113C106
:100AD00007F114C108F115C109F116C10AF117C1D6
:100AE0000BF135C134F147EF0BF00392ABB2AB9889
:100AF000AB88030103EE00F080517F0BE92604C0B0
:100B0000EFFF802B8151805D700BD8A48B82000099
:100B10008051815D700BD8A48B9281518019D8B41B
:100B2000079047EF0BF0F2940101453F47EF0BF0C0
:100B3000462B47EF0BF09E900101533F47EF0BF020
:100B4000542B47EF0BF09E9211B843EF08F00400CE
:100B500066A1ABEF05F08BB4B5EF05F010ACB5EFC7
:100B600005F08B84109CB6EF05F08B94077C07ACE6
:100B7000D1EF05F0C274C2B4CBEF05F0C3CFB7F527
:100B8000C4CFB8F50501D890B833B733D890B8338F
:100B9000B733D2EF05F0C3CF55F1C4CF56F1D2EF42
:100BA00005F0C28207B444EF06F047C14BF148C1DB
:100BB0004CF149C14DF14AC14EF15EC162F15FC1D4
:100BC00063F160C164F161C165F113A8EAEF05F05A
:100BD000138C13989AC1BAF19BC1BBF19CC1BCF1B3
:100BE0009DC1BDF19EC1BEF19FC1BFF1A0C1C0F1C9
:100BF000A1C1C1F1A2C1C2F1A3C1C3F1A4C1C4F199
:100C0000A5C1C5F1A6C1C6F1A7C1C7F1A8C1C8F168
:100C1000A9C1C9F1AAC1CAF1ABC1CBF1ACC1CCF138
:100C2000ADC1CDF1AEC1CEF1AFC1CFF1B0C1D0F108
:100C3000B1C1D1F1B2C1D2F1B3C1D3F1B4C1D4F1D8
:100C4000B5C1D5F1B6C1D6F1B7C1D7F1B8C1D8F1A8
:100C5000B9C1D9F1B7C5B9F5B8C5BAF5B9C5BBF5CC
:100C6000BAC5BCF5010155515B2756515C23E86AB2
:100C70005D230E2E44EF06F05CC157F15DC158F1C3
:100C80005B6B5C6B5D6B078E0201002F47EF0BF017
:100C90003C0E006F1D50E00BE00AE86612881BBE98
:100CA00002D01BB4108E00C10CF101C10DF102C1C4
:100CB0000EF103C10FF104C110F105C111F106C11C
:100CC00012F107C113F108C114F109C115F10AC1EC
:100CD00016F10BC117F134C135F181AAACEF06F062
:100CE00015A4F7EF06F005012F51000AD8B43AEF2A
:100CF00007F005012F51010AD8B4B6EF06F005013F
:100D00002F51020AD8B4F7EF06F005012F51030A5C
:100D1000D8B4F7EF06F005012F51040AD8B4F7EF65
:100D200006F005012F51050AD8B4F7EF06F00501CA
:100D30002F51060AD8B4F7EF06F005012F51070A24
:100D4000D8B4F7EF06F005012F51320AD8B4B4EF4A
:100D500006F02F6B3AEF07F000011650030AD8B4E3
:100D6000F7EF06F03AEF07F03AEF07F005015767A3
:100D7000C1EF06F05867C1EF06F05967C1EF06F002
:100D80005A67C5EF06F03AEF07F05BC500F15CC5A6
:100D900001F15DC502F15EC503F10101010E046FB1
:100DA000000E056F000E066F000E076FB1EC30F0FD
:100DB00000C15BF501C15CF502C15DF503C15EF5E3
:100DC00001010067EBEF06F00167EBEF06F0026749
:100DD000EBEF06F003673AEF07F057C55BF558C530
:100DE0005CF559C55DF55AC55EF524EF07F00FBEF9
:100DF0000CEF07F010A011EF07F00101476708EFB3
:100E000007F0486708EF07F0496708EF07F04A67FF
:100E10000CEF07F011EF07F007AE11EF07F024EF2A
:100E200007F00501312F3AEF07F03C0E316F302FFC
:100E30003AEF07F00101000E626FE00E636FA50E3E
:100E4000646F010E656F138800011650000AD8B454
:100E500032EF07F000011650030AD8B437EF07F05D
:100E60003AEF07F00001010E166E3AEF07F00001AD
:100E7000040E166E0501666B37B740EF07F066810A
:100E80000CC100F10DC101F10EC102F10FC103F15E
:100E900010C104F111C105F112C106F113C107F12E
:100EA00014C108F115C109F116C10AF117C10BF1FE
:100EB00035C134F100C10CF101C10DF102C10EF1D7
:100EC00003C10FF104C110F105C111F106C112F106
:100ED00007C113F108C114F109C115F10AC116F1D6
:100EE0000BC117F134C135F101018E677FEF07F0B7
:100EF0008F677FEF07F090677FEF07F0916783EFD1
:100F000007F0B4EF07F092C100F193C101F194C171
:100F100002F195C103F10101010E046F000E056F8E
:100F2000000E066F000E076FB1EC30F000C192F1B9
:100F300001C193F102C194F103C195F10101006770
:100F4000A9EF07F00167A9EF07F00267A9EF07F023
:100F50000367B4EF07F08EC192F18FC193F190C196
:100F600094F191C195F10F80D57ED5BE6ED0D6CFCC
:100F700047F1D7CF48F145C149F1E86AE8CF4AF1D6
:100F8000138A1CBE02D01CA0108C109047C100F127
:100F900048C101F149C102F14AC103F101010A0E40
:100FA000046F000E056F000E066F000E076FB1ECA8
:100FB00030F003AF1080010154A7EBEF07F00F9A58
:100FC0000F9C0F9E0101000E5E6F600E5F6F3D0E65
:100FD000606F080E616F010147BFFBEF07F04867C4
:100FE000FBEF07F04967FBEF07F04A67FBEF07F0FD
:100FF000F28820EF08F0F2985E6B5F6B606B616BBC
:101000009A6B9B6B9C6B9D6B9E6B9F6BA06BA16B9C
:10101000A26BA36BA46BA56BA66BA76BA86BA96B4C
:10102000AA6BAB6BAC6BAD6BAE6BAF6BB06BB16BFC
:10103000B26BB36BB46BB56BB66BB76BB86BB96BAC
:10104000D76AD66A0101456B466B0CC100F10DC130
:1010500001F10EC102F10FC103F110C104F111C180
:1010600005F112C106F113C107F114C108F115C150
:1010700009F116C10AF117C10BF135C134F147EF7F
:101080000BF047EF0BF00201002FABEF0AF0D59EFB
:10109000D6CF47F1D7CF48F145C149F1E86AE8CF4B
:1010A0004AF1138AD76AD66A0101456B466BD58E21
:1010B0001D50E00BE00AE86612881BBE02D01BB48C
:1010C000108E1AAE1F8C00C10CF101C10DF102C1CE
:1010D0000EF103C10FF104C110F105C111F106C1F8
:1010E00012F107C113F108C114F109C115F10AC1C8
:1010F00016F10BC117F134C135F10FA0109A11B8D8
:101100008DEF08F00101620E046F010E056F000EF5
:10111000066F000E076F96EF08F00101A70E046F2F
:10112000020E056F000E066F000E076F47C100F13B
:1011300048C101F149C102F14AC103F1B1EC30F0FB
:1011400003BFA9EF08F01CBE02D01CA0108C11B088
:101150000F800CC100F10DC101F10EC102F10FC1F0
:1011600003F110C104F111C105F112C106F113C15F
:1011700007F114C108F115C109F116C10AF117C12F
:101180000BF135C134F102013C0E006F00C10CF1CE
:1011900001C10DF102C10EF103C10FF104C110F143
:1011A00005C111F106C112F107C113F108C114F113
:1011B00009C115F10AC116F10BC117F134C135F19E
:1011C00081BAE6EF08F015B225EF09F015A025EF7A
:1011D00009F015A470EF09F005012F51000AD8B4E9
:1011E000B3EF09F005012F51010AD8B42FEF09F030
:1011F00005012F51020AD8B470EF09F005012F51F3
:10120000030AD8B470EF09F005012F51040AD8B4CD
:1012100070EF09F005012F51050AD8B470EF09F0FD
:1012200005012F51060AD8B470EF09F005012F51BE
:10123000070AD8B470EF09F005012F51320AD8B46B
:101240002DEF09F02F6BB3EF09F000011650030AE0
:10125000D8B470EF09F0B3EF09F0B3EF09F005016E
:1012600057673AEF09F058673AEF09F059673AEFD4
:1012700009F05A673EEF09F0B3EF09F05BC500F1E2
:101280005CC501F15DC502F15EC503F10101010E0E
:10129000046F000E056F000E066F000E076FB1ECB5
:1012A00030F000C15BF501C15CF502C15DF503C121
:1012B0005EF50101006764EF09F0016764EF09F072
:1012C000026764EF09F00367B3EF09F057C55BF5F8
:1012D00058C55CF559C55DF55AC55EF59DEF09F039
:1012E0000FBE85EF09F010A08AEF09F001014767F2
:1012F00081EF09F0486781EF09F0496781EF09F054
:101300004A6785EF09F08AEF09F007AE8AEF09F026
:101310009DEF09F00501312FB3EF09F03C0E316F5D
:10132000302FB3EF09F00101000E626FE00E636F22
:10133000A50E646F010E656F138800011650000A38
:10134000D8B4ABEF09F000011650030AD8B4B0EFDF
:1013500009F0B3EF09F00001010E166EB3EF09F0CA
:101360000001040E166E0501666B37B7B9EF09F080
:1013700066810CC100F10DC101F10EC102F10FC176
:1013800003F110C104F111C105F112C106F113C13D
:1013900007F114C108F115C109F116C10AF117C10D
:1013A0000BF135C134F100C10CF101C10DF102C1E5
:1013B0000EF103C10FF104C110F105C111F106C115
:1013C00012F107C113F108C114F109C115F10AC1E5
:1013D00016F10BC117F134C135F101018E67F8EF39
:1013E00009F08F67F8EF09F09067F8EF09F091675F
:1013F000FCEF09F02DEF0AF092C100F193C101F169
:1014000094C102F195C103F10101010E046F000EB8
:10141000056F000E066F000E076FB1EC30F000C1D3
:1014200092F101C193F102C194F103C195F101015F
:10143000006722EF0AF0016722EF0AF0026722EF4D
:101440000AF003672DEF0AF08EC192F18FC193F17C
:1014500090C194F191C195F10F80109047C100F1B6
:1014600048C101F149C102F14AC103F101010A0E6B
:10147000046F000E056F000E066F000E076FB1ECD3
:1014800030F003AF1080010154A753EF0AF00F9A18
:101490000F9C0F9E0101000E5E6F600E5F6F3D0E90
:1014A000606F080E616F47C100F148C101F149C189
:1014B00002F14AC103F10101140E046F050E056F1C
:1014C000000E066F000E076FB1EC30F003AF6CEF4B
:1014D0000AF0F28891EF0AF0F2985E6B5F6B606B36
:1014E000616B9A6B9B6B9C6B9D6B9E6B9F6BA06BF8
:1014F000A16BA26BA36BA46BA56BA66BA76BA86B70
:10150000A96BAA6BAB6BAC6BAD6BAE6BAF6BB06B1F
:10151000B16BB26BB36BB46BB56BB66BB76BB86BCF
:10152000B96B0CC100F10DC101F10EC102F10FC187
:1015300003F110C104F111C105F112C106F113C18B
:1015400007F114C108F115C109F116C10AF117C15B
:101550000BF135C134F104008BB4B6EF0AF010ACD6
:10156000B6EF0AF08B84109CB7EF0AF08B94077CDF
:1015700007ACD2EF0AF0C274C2B4CCEF0AF0C3CF0A
:10158000B7F5C4CFB8F50501D890B833B733D890C4
:10159000B833B733D3EF0AF0C3CF55F1C4CF56F108
:1015A000D3EF0AF0C28207B445EF0BF047C14BF10D
:1015B00048C14CF149C14DF14AC14EF15EC162F1E1
:1015C0005FC163F160C164F161C165F113A8EBEF24
:1015D0000AF0138C13989AC1BAF19BC1BBF19CC15C
:1015E000BCF19DC1BDF19EC1BEF19FC1BFF1A0C1C3
:1015F000C0F1A1C1C1F1A2C1C2F1A3C1C3F1A4C193
:10160000C4F1A5C1C5F1A6C1C6F1A7C1C7F1A8C162
:10161000C8F1A9C1C9F1AAC1CAF1ABC1CBF1ACC132
:10162000CCF1ADC1CDF1AEC1CEF1AFC1CFF1B0C102
:10163000D0F1B1C1D1F1B2C1D2F1B3C1D3F1B4C1D2
:10164000D4F1B5C1D5F1B6C1D6F1B7C1D7F1B8C1A2
:10165000D8F1B9C1D9F1B7C5B9F5B8C5BAF5B9C5A9
:10166000BBF5BAC5BCF5010155515B2756515C234A
:10167000E86A5D230E2E45EF0BF05CC157F15DC1AA
:1016800058F15B6B5C6B5D6B078E47EF0BF002C034
:10169000E0FF005001C0D8FF1000A6B24DEF0BF0E4
:1016A0000CC0A9FF0BC0A8FFA69EA69CA684F29E14
:1016B000550EA76EAA0EA76EA682F28EA694A6B2AB
:1016C0005FEF0BF00C2A1200A96EA69EA69CA680C6
:1016D000A8500C2A120004012C0E826FABEC0EF005
:1016E000C6EC31F00C5064EC0BF0E8CF00F10C507C
:1016F00064EC0BF0E8CF01F101AF84EF0BF00101D6
:10170000FF0E026FFF0E036F4FEC31F0296790EF71
:101710000BF00401200E826FABEC0EF095EF0BF096
:1017200004012D0E826FABEC0EF059EC2FF012007D
:1017300015941596076A0F6A106A116A126A136A7D
:10174000166A0F010E0EC16E860EC06E030EC26EBB
:101750000F01680E896E130E926E080E8A6EF50EDA
:10176000936E8B6A900E946E81A4BBEF0BF09492F3
:10177000949CBDEF0BF09482948CC80E64EC0BF03B
:10178000E8CF25F000012550FE0AD8B4D3EF0BF0C6
:1017900000012550FD0AD8B4D8EF0BF00F0E266ECD
:1017A0008F0E276E09D00E0E266E8E0E276E04D079
:1017B0000D0E266E8D0E276E64EC32F0A4EC33F025
:1017C000F18EF19EFC0E64EC0BF0E8CF0BF00BA059
:1017D00011800BA211820BA411840BA81188C90ED1
:1017E00064EC0BF0E8CF1AF0CA0E64EC0BF0E8CF13
:1017F0001BF0CB0E64EC0BF0E8CF1CF0CC0E64ECCD
:101800000BF0E8CF1DF0FB0E64EC0BF0E8CF38F0E6
:10181000CE0E64EC0BF0E8CF14F0CD0E64EC0BF0C0
:10182000E8CF37F01F6A206A0E6A01015B6B5C6BC0
:101830005D6B576B586BF29A0101476B486B496BB4
:101840004A6B4B6B4C6B4D6B4E6B4F6B506B516BD4
:10185000526B456B466BD76AD66A0F01280ED56E60
:10186000F28A9D90B00ECD6E01015E6B5F6B606B76
:10187000616B626B636B646B656B666B676B686BEC
:10188000696B536B546BCF6ACE6A0F9A0F9C0F9E95
:101890009D80760ECA6E9D8202013C0E006FCC6A5E
:1018A000160E64EC0BF0E8CF00F1170E64EC0BF0B1
:1018B000E8CF01F1180E64EC0BF0E8CF02F1190E3D
:1018C00064EC0BF0E8CF03F1010103AF82EF0CF001
:1018D000C6EC31F0160E0C6E00C10BF04DEC0BF0A7
:1018E000170E0C6E01C10BF04DEC0BF0180E0C6EC8
:1018F00002C10BF04DEC0BF0190E0C6E03C10BF096
:101900004DEC0BF000C18EF101C18FF102C190F1DD
:1019100003C191F100C192F101C193F102C194F1AF
:1019200003C195F11A0E64EC0BF0E8CF00F11B0E29
:1019300064EC0BF0E8CF01F11C0E64EC0BF0E8CF87
:1019400002F11D0E64EC0BF0E8CF03F1010103AFCF
:10195000D8EF0CF0C6EC31F01A0E0C6E00C10BF093
:101960004DEC0BF01B0E0C6E01C10BF04DEC0BF0AF
:101970001C0E0C6E02C10BF04DEC0BF01D0E0C6E2C
:1019800003C10BF04DEC0BF01A0E64EC0BF0E8CF3A
:1019900000F11B0E64EC0BF0E8CF01F11C0E64ECBF
:1019A0000BF0E8CF02F11D0E64EC0BF0E8CF03F171
:1019B00000C196F101C197F102C198F103C199F1FB
:1019C000240EAC6E900EAB6E240EAC6E080EB86E8C
:1019D000000EB06E1F0EAF6E0401806B816B0F01A5
:1019E000900EAB6E0F019D8A0301806B816BC26B01
:1019F0008B9235EC37F035EC37F017EC39F013EC0F
:101A000035F0200E64EC0BF0E8CF2FF505012F51D7
:101A1000FF0AD8A413EF0DF02F6B200E0C6E2FC50C
:101A20000BF04DEC0BF00501010E306F3C0E316FE9
:101A3000250E64EC0BF0E8CF00F1260E64EC0BF001
:101A4000E8CF01F1270E64EC0BF0E8CF02F1280E8D
:101A500064EC0BF0E8CF03F1010103AF4AEF0DF0A6
:101A6000C6EC31F0250E0C6E00C10BF04DEC0BF006
:101A7000260E0C6E01C10BF04DEC0BF0270E0C6E18
:101A800002C10BF04DEC0BF0280E0C6E03C10BF0F5
:101A90004DEC0BF000C157F501C158F502C159F5E5
:101AA00003C15AF500C15BF501C15CF502C15DF5EA
:101AB00003C15EF5290E64EC0BF0E8CF5FF505017C
:101AC00060515F5DD8A05FC560F5210E64EC0BF03E
:101AD000E8CF00F1220E64EC0BF0E8CF01F1230E09
:101AE00064EC0BF0E8CF02F1240E64EC0BF0E8CFCD
:101AF00003F1010103AFABEF0DF0C6EC31F0210EA5
:101B00000C6E00C10BF04DEC0BF0220E0C6E01C1FF
:101B10000BF04DEC0BF0230E0C6E02C10BF04DECF4
:101B20000BF0240E0C6E03C10BF04DEC0BF0210EEC
:101B300064EC0BF0E8CF00F1220E64EC0BF0E8CF80
:101B400001F1230E64EC0BF0E8CF02F1240E64ECFB
:101B50000BF0E8CF03F100C161F501C162F502C1EC
:101B600063F503C164F524EC34F041EC33F077EC19
:101B700032F01590C70E64EC0BF0E8CF00F10101D4
:101B800000B1C6EF0DF01592C7EF0DF0158281AAD6
:101B9000D5EF0DF015B4D0EF0DF01580D5EF0DF0A9
:101BA00056EC39F015A0BFEF39F007900001F28E26
:101BB000F28C12AE03D012BC83EF19F007B0CFEF56
:101BC0002DF00FB0BFEF26F010BEBFEF26F012B819
:101BD000BFEF26F000011650010AD8B4C7EF1DF080
:101BE00081BAFBEF0DF000011650040AD8B440EFA3
:101BF0001CF001EF0EF000011650040AD8B403EFF8
:101C00001EF00301805181197F0BD8B4CFEF2DF066
:101C100013EE00F081517F0BE126812BE7CFE8FF27
:101C2000E00BD8B4CFEF2DF023EE82F0C2513F0B82
:101C3000D926E7CFDFFFC22BDF50780AD8A4CFEF39
:101C40002DF0078092C100F193C101F194C102F11E
:101C500095C103F10101040E046F000E056F000E23
:101C6000066F000E076FB1EC30F000AF41EF0EF0E1
:101C70000101030E926F000E936F000E946F000E21
:101C8000956F03018251720AD8B440EF26F0825159
:101C9000520AD8B440EF26F08251750AD8B440EF0A
:101CA00026F08251680AD8B4BFEF0EF08251630A61
:101CB000D8B489EF2AF08251690AD8B40DEF21F027
:101CC00082517A0AD8B420EF22F08251490AD8B45E
:101CD000ACEF20F08251500AD8B4CAEF1FF0825105
:101CE000700AD8B40DEF20F08251540AD8B438EFFE
:101CF00020F08251740AD8B47EEF20F08251410A5C
:101D0000D8B4C4EF0FF082514B0AD8B4C1EF0EF033
:101D100082516D0AD8B434EF14F082514D0AD8B410
:101D20004DEF14F08251730AD8B470EF25F0825150
:101D3000530AD8B4D5EF25F082514C0AD8B4DCEF61
:101D400014F08251590AD8B485EF13F012AE01D0C5
:101D5000128CC0EF2AF0040114EE00F080517F0BCA
:101D6000E12682C4E7FF802B120004010D0E826F72
:101D7000ABEC0EF00A0E826FABEC0EF01200BEEF71
:101D80002AF004014B0E826FABEC0EF004012C0E16
:101D9000826FABEC0EF081B802D037B630D00301C1
:101DA0008351430AD8B406EF0FF003018351630A4D
:101DB000D8B408EF0FF003018351520AD8B40AEFE8
:101DC0000FF003018351720AD8B40CEF0FF0030136
:101DD0008351470AD8B40EEF0FF003018351670A0D
:101DE000D8B410EF0FF003018351540AD8B412EFA6
:101DF0000FF003018351740AD8B482EF0FF003018E
:101E00008351550AD8B414EF0FF083D037807BD0BC
:101E1000379079D0378277D0379275D0378473D0A6
:101E2000379471D037866FD084C330F185C331F1D8
:101E300086C332F187C333F10101296B14EC32F010
:101E40008BEC31F000C104F101C105F102C106F1D2
:101E500003C107F107EC32F0200EF86EF76AF66A5C
:101E60000900F5CF2CF10900F5CF2DF10900F5CFD0
:101E70002EF10900F5CF2FF10900F5CF30F109005F
:101E8000F5CF31F10900F5CF32F10900F5CF33F18B
:101E90000101296B14EC32F08BEC31F0B1EC30F035
:101EA000010100675BEF0FF001675BEF0FF0026766
:101EB0005BEF0FF0036701D025D004014E0E826F57
:101EC000ABEC0EF004016F0E826FABEC0EF0040170
:101ED0004D0E826FABEC0EF00401610E826FABEC25
:101EE0000EF00401740E826FABEC0EF00401630E71
:101EF000826FABEC0EF00401680E826FABEC0EF05B
:101F0000BEEF2AF03796CD0E0C6E37C00BF04DECBD
:101F10000BF0CD0E64EC0BF0E8CF37F037B006D005
:101F20000401630E826FABEC0EF005D00401430E8A
:101F3000826FABEC0EF037B206D00401720E826FE6
:101F4000ABEC0EF005D00401520E826FABEC0EF03C
:101F500037B406D00401670E826FABEC0EF005D0EB
:101F60000401470E826FABEC0EF037B606D00401C9
:101F7000740E826FABEC0EF005D00401540E826F2C
:101F8000ABEC0EF0BEEF2AF00401410E826FABEC19
:101F90000EF003018351310AD8B4A5EF12F003010A
:101FA0008351320AD8B4D5EF11F003018351330ABB
:101FB000D8B45EEF11F003018351340AD8B44EEF68
:101FC00010F003018351350AD8B4EEEF0FF004018D
:101FD0003F0E826FABEC0EF0BEEF2AF0030184518E
:101FE000300AD8B414EF10F003018451310AD8B488
:101FF00017EF10F003018451650AD8B408EF10F010
:1020000003018451640AD8B40BEF10F018EF10F0FC
:1020100038900CEF10F03880FB0E0C6E38C00BF0CF
:102020004DEC0BF018EF10F08B9018EF10F08B8048
:102030000401350E826FABEC0EF004012C0E826FA2
:10204000ABEC0EF08BB02CEF10F00401300E826F71
:10205000ABEC0EF031EF10F00401310E826FABECFF
:102060000EF004012C0E826FABEC0EF0FB0E64EC54
:102070000BF0E8CF38F038A045EF10F00401640E03
:10208000826FABEC0EF04AEF10F00401650E826F28
:10209000ABEC0EF04CEF10F0BEEF2AF0CC0E64EC7F
:1020A0000BF0E8CF0BF004012C0E826FABEC0EF0BE
:1020B00003018451310AD8B472EF10F00301845146
:1020C000300AD8B474EF10F0030184514D0AD8B42B
:1020D0007EEF10F003018451540AD8B485EF10F05C
:1020E0009CEF10F08A8401D08A940BAE04D00BAC24
:1020F00002D00BBA21D0E00E0B1218D01F0E0B1617
:102100008539E844E00B0B1211D0E00E0B1607ECFA
:1021100032F085C332F186C333F10101296B14EC2F
:1021200032F08BEC31F000511F0B0B12CC0E0C6E09
:102130000BC00BF04DEC0BF00401340E826FABECD6
:102140000EF004012C0E826FABEC0EF0CC0E64ECA2
:102150000BF0E8CF1DF08AB406D00401300E826F78
:10216000ABEC0EF005D00401310E826FABEC0EF03B
:1021700004012C0E826FABEC0EF01D38E840070B0B
:10218000E8CF82F40401300E8227ABEC0EF004019C
:102190002C0E826FABEC0EF0C6EC31F01D501F0B15
:1021A000E8CF00F14FEC31F032C182F40401300E7F
:1021B0008227ABEC0EF033C182F40401300E82278B
:1021C000ABEC0EF004012C0E826FABEC0EF0C6EC03
:1021D00031F031C000F100AF0BD0FF0E016FFF0EE8
:1021E000026FFF0E036F04012D0E826FABEC0EF039
:1021F0004FEC31F031C182F40401300E8227ABEC98
:102200000EF032C182F40401300E8227ABEC0EF0E6
:1022100033C182F40401300E8227ABEC0EF00401CE
:102220002C0E826FABEC0EF0C6EC31F030C000F13A
:102230004FEC31F031C182F40401300E8227ABEC57
:102240000EF032C182F40401300E8227ABEC0EF0A6
:1022500033C182F40401300E8227ABEC0EF004018E
:102260002C0E826FABEC0EF0C6EC31F032C000F1F8
:1022700000AF0BD0FF0E016FFF0E026FFF0E036F5A
:1022800004012D0E826FABEC0EF04FEC31F031C13A
:1022900082F40401300E8227ABEC0EF032C182F4DE
:1022A0000401300E8227ABEC0EF033C182F404013E
:1022B000300E8227ABEC0EF0BEEF2AF0CB0E64ECB2
:1022C0000BF0E8CF0BF004012C0E826FABEC0EF09C
:1022D00003018451450AD8B482EF11F003018451FF
:1022E000440AD8B485EF11F003018451300AD8B400
:1022F00088EF11F003018451310AD8B48CEF11F04A
:1023000097EF11F00B9E91EF11F00B8E91EF11F002
:10231000FC0E0B1691EF11F0FC0E0B160B8091EFDB
:1023200011F0CB0E0C6E0BC00BF04DEC0BF004015A
:10233000330E826FABEC0EF004012C0E826FABEC0F
:102340000EF0CB0E64EC0BF0E8CF1CF01CBEB0EF2F
:1023500011F00401450E826FABEC0EF0B5EF11F0F9
:102360000401440E826FABEC0EF004012C0E826F60
:10237000ABEC0EF00401300E826FABEC0EF00401FA
:102380002C0E826FABEC0EF01CB0CEEF11F00401FE
:10239000300E826FABEC0EF0D3EF11F00401310E72
:1023A000826FABEC0EF0BEEF2AF0CA0E64EC0BF0BD
:1023B000E8CF0BF004012C0E826FABEC0EF00301A2
:1023C0008451450AD8B411EF12F003018451440A34
:1023D000D8B414EF12F0030184514D0AD8B41DEFA4
:1023E00012F003018451410AD8B417EF12F003012F
:1023F0008451460AD8B41AEF12F003018451560AE8
:10240000D8B425EF12F003018451500AD8B430EF4C
:1024100012F003018451520AD8B433EF12F03CEFAA
:1024200012F00B9E36EF12F00B8E36EF12F00B9C73
:1024300036EF12F00B8C36EF12F0FC0E0B1685C344
:10244000E8FF030B0B1236EF12F0C70E0B1685C315
:10245000E8FF070BE846E846E8460B1236EF12F0B5
:102460000B8436EF12F00B9436EF12F0CA0E0C6E9E
:102470000BC00BF04DEC0BF0CA0E64EC0BF0E8CF88
:102480001BF00401320E826FABEC0EF004012C0E37
:10249000826FABEC0EF01BBE55EF12F00401450E3F
:1024A000826FABEC0EF05AEF12F00401440E826F13
:1024B000ABEC0EF004012C0E826FABEC0EF01BC0E7
:1024C000E8FF030BE8CF82F40401300E8227ABEC67
:1024D0000EF004012C0E826FABEC0EF01BBC78EFFB
:1024E00012F00401410E826FABEC0EF07DEF12F0A2
:1024F0000401460E826FABEC0EF004012C0E826FCD
:10250000ABEC0EF01BC0E8FF380BE842E842E842B3
:10251000E8CF82F40401300E8227ABEC0EF0040108
:102520002C0E826FABEC0EF01BB49EEF12F0040188
:10253000520E826FABEC0EF0A3EF12F00401500EBE
:10254000826FABEC0EF0BEEF2AF0C90E64EC0BF01C
:10255000E8CF0BF004012C0E826FABEC0EF0030100
:102560008451450AD8B4C3EF12F003018451440AE0
:10257000D8B4C6EF12F0030184514D0AD8B4C9EFA4
:1025800012F0D7EF12F00B9ED1EF12F00B8ED1EFBD
:1025900012F0F80E0B1685C3E8FF070B0B12D1EFF4
:1025A00012F0C90E0C6E0BC00BF04DEC0BF00401D9
:1025B000310E826FABEC0EF004012C0E826FABEC8F
:1025C0000EF0C90E64EC0BF0E8CF1AF01ABE06D07C
:1025D0000401450E826FABEC0EF005D00401440EF1
:1025E000826FABEC0EF004012C0E826FABEC0EF0A0
:1025F0001AC0E8FF070BE8CF82F40401300E8227EF
:10260000ABEC0EF004012C0E826FABEC0EF00780E9
:10261000C6EC31F02CC0E8FF003B00430043030B45
:102620004FEC31F033C182F40401300E8227ABEC61
:102630000EF004012C0E826FABEC0EF0C6EC31F004
:102640002CC001F1019F019D2DC000F101014FEC53
:1026500031F02FC182F40401300E8227ABEC0EF072
:1026600030C182F40401300E8227ABEC0EF031C190
:1026700082F40401300E8227ABEC0EF032C182F4FA
:102680000401300E8227ABEC0EF033C182F404015A
:10269000300E8227ABEC0EF004012C0E826FABECF7
:1026A0000EF0C6EC31F02EC001F12FC000F1D89031
:1026B00001330033D8900133003301014FEC31F086
:1026C0002FC182F40401300E8227ABEC0EF030C132
:1026D00082F40401300E8227ABEC0EF031C182F49B
:1026E0000401300E8227ABEC0EF032C182F40401FB
:1026F000300E8227ABEC0EF033C182F40401300EB1
:102700008227ABEC0EF0BEEF2AF0FC0E64EC0BF06F
:10271000E8CF0BF003018351520AD8B4BCEF13F099
:1027200003018351720AD8B4BFEF13F00301835140
:10273000500AD8B4C2EF13F003018351700AD8B421
:10274000C5EF13F003018351550AD8B4C8EF13F055
:1027500003018351750AD8B4CBEF13F00301835101
:10276000430AD8B4D4EF13F003018351630AD8B4F9
:10277000D7EF13F0E0EF13F00B90DAEF13F00B80CC
:10278000DAEF13F00B92DAEF13F00B82DAEF13F0BB
:102790000B94DAEF13F00B84DAEF13F00B96DAEF09
:1027A00013F00B86DAEF13F00B98DAEF13F00B88C7
:1027B000DAEF13F0FC0E0C6E0BC00BF04DEC0BF0CF
:1027C0000401590E826FABEC0EF01190119211942E
:1027D0001198FC0E64EC0BF0E8CF0BF00BA011800D
:1027E0000BA211820BA411840BA8118811A000EF79
:1027F00014F00401520E826FABEC0EF005EF14F0F2
:102800000401720E826FABEC0EF011A80FEF14F002
:102810000401430E826FABEC0EF014EF14F00401D0
:10282000630E826FABEC0EF011A21EEF14F00401E8
:10283000500E826FABEC0EF023EF14F00401700E1B
:10284000826FABEC0EF011A42DEF14F00401550EC5
:10285000826FABEC0EF032EF14F00401750E826F54
:10286000ABEC0EF0BEEF2AF004016D0E826FABEC04
:102870000EF003018351300AD8B48CEF14F0030139
:102880008351310AD8B49FEF14F003018351320A07
:10289000D8B4B2EF14F0C0EF2AF004014D0E826FED
:1028A000ABEC0EF007EC32F084C331F185C332F1AA
:1028B00086C333F10101296B14EC32F08BEC31F05B
:1028C00003018351300AD8B474EF14F0030183512B
:1028D000310AD8B47CEF14F003018351320AD8B422
:1028E00084EF14F0C0EF2AF0FD0E0C6E00C10BF067
:1028F0004DEC0BF08CEF14F0FE0E0C6E00C10BF0E3
:102900004DEC0BF09FEF14F0FF0E0C6E00C10BF0BE
:102910004DEC0BF0B2EF14F00401300E826FABEC13
:102920000EF004012C0E826FABEC0EF0C6EC31F011
:10293000FD0E64EC0BF0E8CF00F1C3EF14F00401DE
:10294000310E826FABEC0EF004012C0E826FABECFB
:102950000EF0C6EC31F0FE0E64EC0BF0E8CF00F1A7
:10296000C3EF14F00401320E826FABEC0EF0C6EC34
:1029700031F004012C0E826FABEC0EF0FF0E64EC14
:102980000BF0E8CF00F14FEC31F031C182F40401DB
:10299000300E8227ABEC0EF032C182F40401300E0F
:1029A0008227ABEC0EF033C182F40401300E822793
:1029B000ABEC0EF0BEEF2AF003018351300AD8B41D
:1029C00030EF1AF003018351310AD8B46EEF1BF0D7
:1029D00003018351320AD8B4DCEF1BF003018351A9
:1029E000330AD8B4ECEF1BF003018351340AD8B496
:1029F00047EF1CF003018351350AD8B41BEF1EF0DA
:102A000003018351360AD8B449EF1EF00301835104
:102A1000370AD8B408EF18F003018351380AD8B444
:102A2000A6EF18F003018351440AD8B434EF16F02E
:102A300003018351640AD8B454EF16F003018351A3
:102A4000460AD8B420EF1DF0030183514D0AD8B4D3
:102A500081EF16F0030183516D0AD8B49BEF16F095
:102A6000030183515A0AD8B4E8EF1AF003018351E5
:102A7000490AD8B449EF1FF003018351500AD8B472
:102A80007BEF1EF003018351540AD8B4F4EF1EF01B
:102A900003018351630AD8B4BBEF16F003018351DD
:102AA000430AD8B4B3EF17F003018351730AD8B4C3
:102AB000B9EF16F003018351610AD8B481EF15F024
:102AC00003018351650AD8B480EF1AF003018351E2
:102AD000450AD8B48EEF1AF003018351620AD8B4C4
:102AE0009CEF1AF003018351420AD8B4AAEF1AF0FE
:102AF00003018351760AD8B4B8EF1AF0D8A4C0EF16
:102B00002AF004014C0E826FABEC0EF00401610E52
:102B1000826FABEC0EF041EC33F004012C0E826FAF
:102B2000ABEC0EF0C6EC31F0AFC500F101014FEC9B
:102B300031F031C182F40401300E8227ABEC0EF08B
:102B400032C182F40401300E8227ABEC0EF033C1A7
:102B500082F40401300E8227ABEC0EF004012C0E3F
:102B6000826FABEC0EF0C6EC31F0B0C500F10101A4
:102B70004FEC31F031C182F40401300E8227ABEC0E
:102B80000EF032C182F40401300E8227ABEC0EF05D
:102B900033C182F40401300E8227ABEC0EF0040145
:102BA0002C0E826FABEC0EF0C6EC31F0B1C500F12B
:102BB00001014FEC31F031C182F40401300E822763
:102BC000ABEC0EF032C182F40401300E8227ABEC84
:102BD0000EF033C182F40401300E8227ABEC0EF00C
:102BE00004012C0E826FABEC0EF0C6EC31F0B2C5D6
:102BF00000F101014FEC31F031C182F40401300EDB
:102C00008227ABEC0EF032C182F40401300E822731
:102C1000ABEC0EF033C182F40401300E8227ABEC32
:102C20000EF004012C0E826FABEC0EF0C6EC31F00E
:102C3000B6C500F101014FEC31F031C182F404015D
:102C4000300E8227ABEC0EF032C182F40401300E5C
:102C50008227ABEC0EF033C182F40401300E8227E0
:102C6000ABEC0EF077EF1EF003018451300AD8B4BC
:102C700040EF16F003018451310AD8B444EF16F046
:102C80001592159645EF16F01582C70E64EC0BF001
:102C9000E8CF00F10101008115A20091C70E0C6E72
:102CA00000C10BF04DEC0BF0C70E64EC0BF0E8CF5D
:102CB00000F1010100B160EF16F0159261EF16F01E
:102CC000158204014C0E826FABEC0EF00401640E11
:102CD000826FABEC0EF004012C0E826FABEC0EF0A9
:102CE00015B27AEF16F00401300E826FABEC0EF0E5
:102CF0007FEF16F00401310E826FABEC0EF0BEEFE9
:102D00002AF007EC32F084C333F114EC32F08BEC90
:102D100031F0200E0C6E00C10BF04DEC0BF000C139
:102D20002FF505012F51000A06E005012F51010A78
:102D300002E0A4EC33F004014C0E826FABEC0EF019
:102D400004014D0E826FABEC0EF004012C0E826F6D
:102D5000ABEC0EF0C6EC31F02FC500F14FEC31F0CA
:102D600033C182F40401300E8227ABEC0EF077EF12
:102D70001EF0BFEF39F004014C0E826FABEC0EF089
:102D80000401630E826FABEC0EF077EC32F00401BD
:102D90002C0E826FABEC0EF0D0EC16F077EF1EF03D
:102DA000C6EC31F0B5C500F10101003B0F0E001774
:102DB0004FEC31F033C182F40401300E8227ABECCA
:102DC0000EF0B5C500F101010F0E010100174FEC27
:102DD00031F033C182F40401300E8227ABEC0EF0E7
:102DE00004012D0E826FABEC0EF0B4C500F10101B1
:102DF000003B0F0E00174FEC31F033C182F4040199
:102E0000300E8227ABEC0EF0B4C500F101010F0EBD
:102E1000010100174FEC31F033C182F40401300E90
:102E20008227ABEC0EF004012D0E826FABEC0EF09E
:102E3000B3C500F10101003B0F0E00174FEC31F05C
:102E400033C182F40401300E8227ABEC0EF0B3C51F
:102E500000F101010F0E010100174FEC31F033C1F9
:102E600082F40401300E8227ABEC0EF00401200E38
:102E7000826FABEC0EF0B2C500F10F0E010100172E
:102E80004FEC31F033C182F40401300E8227ABECF9
:102E90000EF00401200E826FABEC0EF0B1C500F114
:102EA00001010101003B0F0E00174FEC31F033C15F
:102EB00082F40401300E8227ABEC0EF0B1C500F1B4
:102EC00001010F0E010100174FEC31F033C182F404
:102ED0000401300E8227ABEC0EF004013A0E826F33
:102EE000ABEC0EF0B0C500F10101003B0F0E001776
:102EF0004FEC31F033C182F40401300E8227ABEC89
:102F00000EF0B0C500F101010F0E010100174FECEA
:102F100031F033C182F40401300E8227ABEC0EF0A5
:102F200004013A0E826FABEC0EF0AFC500F1010167
:102F3000003B0F0E00174FEC31F033C182F4040157
:102F4000300E8227ABEC0EF0AFC500F101010F0E81
:102F500000174FEC31F033C182F40401300E8227A8
:102F6000ABEC0EF0120084C3E8FF0F0BE83AE8CF99
:102F7000B5F585C3E8FF0F0B0501B51387C3E8FF5F
:102F80000F0BE83AE8CFB4F588C3E8FF0F0B050153
:102F9000B4138AC3E8FF0F0BE83AE8CFB3F58BC34D
:102FA000E8FF0F0B0501B3138DC3E8FF0F0BE8CF4C
:102FB000B2F58FC3E8FF0F0BE83AE8CFB1F590C345
:102FC000E8FF0F0B0501B11392C3E8FF0F0BE83ABE
:102FD000E8CFB0F593C3E8FF0F0B0501B01395C31D
:102FE000E8FF0F0BE83AE8CFAFF596C3E8FF0F0B09
:102FF0000501AF13E3EC32F004014C0E826FABEC31
:103000000EF00401430E826FABEC0EF0C5EF16F02C
:10301000078404014C0E826FABEC0EF00401370EF6
:10302000826FABEC0EF004012C0E826FABEC0EF055
:1030300005012E51130A06E005012E51170A0DE075
:10304000A3EF18F00101000E006F000E016F100ECB
:10305000026F000E036F36EF18F00101000E006FD3
:10306000000E016F000E026F010E036F4FEC31F086
:103070002AC182F40401300E8227ABEC0EF02BC182
:1030800082F40401300E8227ABEC0EF02CC182F4E6
:103090000401300E8227ABEC0EF02DC182F4040146
:1030A000300E8227ABEC0EF02EC182F40401300EFC
:1030B0008227ABEC0EF02FC182F40401300E822780
:1030C000ABEC0EF030C182F40401300E8227ABEC81
:1030D0000EF031C182F40401300E8227ABEC0EF009
:1030E00032C182F40401300E8227ABEC0EF033C102
:1030F00082F40401300E8227ABEC0EF004012C0E9A
:10310000826FABEC0EF00101200E006F000E016F1C
:10311000000E026F000E036F4FEC31F031C182F4EC
:103120000401300E8227ABEC0EF032C182F40401B0
:10313000300E8227ABEC0EF033C182F40401300E66
:103140008227ABEC0EF0079477EF1EF00501216BA0
:10315000226B236B246B04014C0E826FABEC0EF0E0
:103160000401380E826FABEC0EF004012C0E826F5E
:10317000ABEC0EF00101200E006F000E016F000E8F
:10318000026F000E036F4FEC31F02AC182F404018C
:10319000300E8227ABEC0EF02BC182F40401300E0E
:1031A0008227ABEC0EF02CC182F40401300E822792
:1031B000ABEC0EF02DC182F40401300E8227ABEC93
:1031C0000EF02EC182F40401300E8227ABEC0EF01B
:1031D0002FC182F40401300E8227ABEC0EF030C117
:1031E00082F40401300E8227ABEC0EF031C182F480
:1031F0000401300E8227ABEC0EF032C182F40401E0
:10320000300E8227ABEC0EF033C182F40401300E95
:103210008227ABEC0EF004012C0E826FABEC0EF0AB
:1032200025C500F126C501F127C502F128C503F126
:103230000101200E046F000E056F000E066F000ED8
:10324000076FE2EC30F000C133F501C134F502C183
:1032500035F503C136F54FEC31F02AC182F4040193
:10326000300E8227ABEC0EF02BC182F40401300E3D
:103270008227ABEC0EF02CC182F40401300E8227C1
:10328000ABEC0EF02DC182F40401300E8227ABECC2
:103290000EF02EC182F40401300E8227ABEC0EF04A
:1032A0002FC182F40401300E8227ABEC0EF030C146
:1032B00082F40401300E8227ABEC0EF031C182F4AF
:1032C0000401300E8227ABEC0EF032C182F404010F
:1032D000300E8227ABEC0EF033C182F40401300EC5
:1032E0008227ABEC0EF0B5EC0EF00501336780EFF2
:1032F00019F0346780EF19F0356780EF19F0366701
:1033000002D01FEF1AF0129E129C21C500F122C5B7
:1033100001F123C502F124C503F1899A400EC76E5D
:10332000200EC66E9E96C69E0B0EC96EFF0E9EB6F2
:1033300002D0E82EFCD79E96C69E02C1C9FFFF0EA2
:103340009EB602D0E82EFCD79E96C69E01C1C9FF4C
:10335000FF0E9EB602D0E82EFCD79E96C69E00C1F8
:10336000C9FFFF0E9EB602D0E82EFCD79E96C69EE1
:10337000C952FF0E9EB602D0E82EFCD70501200EE2
:10338000326F040114EE00F080517F0BE1269E960F
:10339000C69EC952FF0E9EB602D0E82EFCD7C9CFFA
:1033A000E7FF0401802B0501322FC1EF19F0898A54
:1033B00033C500F134C501F135C502F136C503F15D
:1033C0000101010E046F000E056F000E066F000E66
:1033D000076FB1EC30F000C133F501C134F502C123
:1033E00035F503C136F505013367FEEF19F0346793
:1033F000FEEF19F03567FEEF19F0366702D01FEFC8
:103400001AF021C500F122C501F123C502F124C53E
:1034100003F10101200E046F000E056F000E066F10
:10342000000E076FB6EC30F000C121F501C122F5A6
:1034300002C123F503C124F5128EC0EF2AF0040166
:10344000450E826FABEC0EF004014F0E826FABECB9
:103450000EF00401460E826FABEC0EF077EF1EF01B
:10346000078417EC39F0C6EC31F02DC500F14FECB4
:1034700031F004014C0E826FABEC0EF00401300E03
:10348000826FABEC0EF004012C0E826FABEC0EF0F1
:1034900031C182F40401300E8227ABEC0EF032C150
:1034A00082F40401300E8227ABEC0EF033C182F4BB
:1034B0000401300E8227ABEC0EF004012C0E826F5B
:1034C000ABEC0EF0C6EC31F02EC500F14FEC31F054
:1034D00031C182F40401300E8227ABEC0EF032C110
:1034E00082F40401300E8227ABEC0EF033C182F47B
:1034F0000401300E8227ABEC0EF0079477EF1EF03C
:1035000004014C0E826FABEC0EF00401650E826F6D
:10351000ABEC0EF0B7EC34F077EF1EF004014C0E7C
:10352000826FABEC0EF00401450E826FABEC0EF037
:10353000CEEC34F077EF1EF004014C0E826FABEC52
:103540000EF00401620E826FABEC0EF0FCEC34F076
:1035500077EF1EF004014C0E826FABEC0EF004010D
:10356000420E826FABEC0EF0E5EC34F077EF1EF01C
:1035700004014C0E826FABEC0EF00401760E826FEC
:10358000ABEC0EF004012C0E826FABEC0EF00001E0
:103590002550FE0AD8B4DAEF1AF000012550FD0AD2
:1035A000D8B4E1EF1AF00401300E826FABEC0EF0EC
:1035B00077EF1EF00401310E826FABEC0EF077EF67
:1035C0001EF00401320E826FABEC0EF077EF1EF0AE
:1035D00004014C0E826FABEC0EF004015A0E826FA8
:1035E000ABEC0EF004012C0E826FABEC0EF017EC7E
:1035F00039F0C6EC31F005012E51130A06E0050141
:103600002E51170A0DE019EF1BF00101000E006F9B
:10361000000E016F100E026F000E036F19EF1BF00A
:103620000101000E006F000E016F000E026F010E0F
:10363000036F0101200E046F000E056F000E066F70
:10364000000E076FE2EC30F04FEC31F02AC182F44B
:103650000401300E8227ABEC0EF02BC182F4040182
:10366000300E8227ABEC0EF02CC182F40401300E38
:103670008227ABEC0EF02DC182F40401300E8227BC
:10368000ABEC0EF02EC182F40401300E8227ABECBD
:103690000EF02FC182F40401300E8227ABEC0EF045
:1036A00030C182F40401300E8227ABEC0EF031C140
:1036B00082F40401300E8227ABEC0EF032C182F4AA
:1036C0000401300E8227ABEC0EF033C182F404010A
:1036D000300E8227ABEC0EF077EF1EF0078404016A
:1036E0004C0E826FABEC0EF00401310E826FABEC2E
:1036F0000EF004012C0E826FABEC0EF025C500F12C
:1037000026C501F127C502F128C503F10101200EEC
:10371000046F000E056F000E066F000E076FE2ECDF
:1037200030F04FEC31F02AC182F40401300E8227D0
:10373000ABEC0EF02BC182F40401300E8227ABEC0F
:103740000EF02CC182F40401300E8227ABEC0EF097
:103750002DC182F40401300E8227ABEC0EF02EC195
:1037600082F40401300E8227ABEC0EF02FC182F4FC
:103770000401300E8227ABEC0EF030C182F404015C
:10378000300E8227ABEC0EF031C182F40401300E12
:103790008227ABEC0EF032C182F40401300E822796
:1037A000ABEC0EF033C182F40401300E8227ABEC97
:1037B0000EF0079477EF1EF0078404014C0E826F21
:1037C000ABEC0EF00401320E826FABEC0EF0EBECC2
:1037D00036F0079477EF1EF0078438B0F2EF1BF055
:1037E00005EF1CF0010E166E04014C0E826FABEC5F
:1037F0000EF00401330E826FABEC0EF048EC37F0A4
:10380000000E166E079479EF1BF0020E166E48EC50
:1038100037F08B800501010E306F3C0E316F0101D6
:103820005E6B5F6B606B616B626B636B646B656B34
:10383000666B676B686B696B536B546BCF6ACE6A50
:103840000F9A0F9C0F9E030E166E04014C0E826F92
:10385000ABEC0EF00401330E826FABEC0EF0040102
:103860002C0E826FABEC0EF004012D0E826FABECD0
:103870000EF00401310E826FABEC0EF0BEEF2AF0B9
:1038800048EC37F0000E166E8B90C0EF2AF00784DC
:1038900004014C0E826FABEC0EF00401340E826F0B
:1038A000ABEC0EF004012C0E826FABEC0EF007ECCB
:1038B00032F084C32AF185C32BF186C32CF187C370
:1038C0002DF188C32EF189C32FF18AC330F18BC348
:1038D00031F18CC332F18DC333F10101296B14EC4A
:1038E00032F08BEC31F0200E046F000E056F000EED
:1038F000066F000E076FC2EC30F000C121F501C168
:1039000022F502C123F503C124F5CAEC38F038C50D
:10391000AFF539C5B0F53AC5B1F53BC5B2F53CC513
:10392000B3F53DC5B4F53EC5B5F5D0EC16F00401D0
:103930002C0E826FABEC0EF03FC500F140C501F1DB
:1039400041C502F142C503F10101000E046F000EF2
:10395000056F010E066F000E076FE2EC30F04FECC2
:1039600031F02967B6EF1CF0BBEF1CF004012D0EFF
:10397000826FABEC0EF030C182F40401300E82276E
:10398000ABEC0EF031C182F40401300E8227ABECB7
:103990000EF004012E0E826FABEC0EF032C182F4F9
:1039A0000401300E8227ABEC0EF033C182F4040127
:1039B000300E8227ABEC0EF004012C0E826FABECC4
:1039C0000EF0C6EC31F043C500F144C501F1EAEC5C
:1039D0002BF004012C0E826FABEC0EF0C6EC31F034
:1039E00045C500F14FEC31F031C182F40401300ED5
:1039F0008227ABEC0EF032C182F40401300E822734
:103A0000ABEC0EF033C182F40401300E8227ABEC34
:103A10000EF004012C0E826FABEC0EF037C5E8FF00
:103A2000E8B806D00401300E826FABEC0EF005D082
:103A30000401310E826FABEC0EF0079477EF1EF0AD
:103A400007EC32F085C32AF186C32BF187C32CF132
:103A500088C32DF189C32EF18AC32FF18BC330F1B6
:103A60008CC331F18DC332F18EC333F10101296B67
:103A700014EC32F08BEC31F00101010E046F000EFA
:103A8000056F000E066F000E076FB1EC30F0100EE0
:103A9000046F000E056F000E066F000E076FC2EC7C
:103AA00030F000C129F501C12AF502C12BF503C18F
:103AB0002CF572EC36F004014C0E826FABEC0EF07C
:103AC0000401460E826FABEC0EF004012C0E826FE7
:103AD000ABEC0EF025C500F126C501F127C502F1BA
:103AE00028C503F10101100E046F000E056F000ED2
:103AF000066F000E076FE2EC30F04FEC31F02AC198
:103B000082F40401300E8227ABEC0EF02BC182F45C
:103B10000401300E8227ABEC0EF02CC182F40401BC
:103B2000300E8227ABEC0EF02DC182F40401300E72
:103B30008227ABEC0EF02EC182F40401300E8227F6
:103B4000ABEC0EF02FC182F40401300E8227ABECF7
:103B50000EF030C182F40401300E8227ABEC0EF07F
:103B600031C182F40401300E8227ABEC0EF032C179
:103B700082F40401300E8227ABEC0EF033C182F4E4
:103B80000401300E8227ABEC0EF077EF1EF038B058
:103B9000CCEF1DF0020E166E48EC37F00001165007
:103BA000020AD8B4EAEF1DF005012F51010AD8B47A
:103BB000E0EF1DF015B2E5EF1DF081BAE5EF1DF065
:103BC000000E166E1584C0EF2AF0050E166E1584D1
:103BD000BFEF39F08B8001015E6B5F6B606B616BD7
:103BE000626B636B646B656B666B676B686B696B51
:103BF000536B546BCF6ACE6A0F9A0F9C0F9E030EC5
:103C0000166EC0EF2AF048EC37F005012F51010A7B
:103C1000D8B411EF1EF015B216EF1EF081BA16EFF0
:103C20001EF0000E166E1584C0EF2AF0050E166EFB
:103C30001584BFEF39F004014C0E826FABEC0EF02F
:103C40000401350E826FABEC0EF004012C0E826F76
:103C5000ABEC0EF0C6EC31F00784B9C500F1079467
:103C60004FEC31F031C182F40401300E8227ABEC0D
:103C70000EF032C182F40401300E8227ABEC0EF05C
:103C800033C182F40401300E8227ABEC0EF077EFE3
:103C90001EF00BEC37F0C6EC31F037C500F14FECFD
:103CA00031F004014C0E826FABEC0EF00401360EC5
:103CB000826FABEC0EF004012C0E826FABEC0EF0B9
:103CC00031C182F40401300E8227ABEC0EF032C118
:103CD00082F40401300E8227ABEC0EF033C182F483
:103CE0000401300E8227ABEC0EF077EF1EF0B5EC3E
:103CF0000EF0C0EF2AF004014C0E826FABEC0EF018
:103D00000401500E826FABEC0EF004012C0E826F9A
:103D1000ABEC0EF085C32AF186C32BF187C32CF1DF
:103D200088C32DF189C32EF18AC32FF18BC330F1E3
:103D30008CC331F18DC332F18EC333F1010114EC28
:103D400032F08BEC31F003018451530A0DE0030192
:103D500084514D0A38E00401780E826FABEC0EF00E
:103D6000B5EC0EF0C0EF2AF00401530E826FABECFD
:103D70000EF0250E0C6E00C10BF04DEC0BF0260E74
:103D80000C6E01C10BF04DEC0BF0270E0C6E02C156
:103D90000BF04DEC0BF0280E0C6E03C10BF04DEC4C
:103DA0000BF000C157F501C158F502C159F503C127
:103DB0005AF500C15BF501C15CF502C15DF503C1B7
:103DC0005EF558EF1FF004014D0E826FABEC0EF064
:103DD000290E0C6E00C10BF04DEC0BF000C15FF52D
:103DE00000C160F558EF1FF004014C0E826FABEC80
:103DF0000EF00401540E826FABEC0EF004012C0E99
:103E0000826FABEC0EF084C32AF185C32BF186C31D
:103E10002CF187C32DF188C32EF189C32FF18AC3FA
:103E200030F18BC331F18DC332F18EC333F1010117
:103E300014EC32F08BEC31F00101000E046F000E37
:103E4000056F010E066F000E076FC2EC30F0210EF9
:103E50000C6E00C10BF04DEC0BF0220E0C6E01C18C
:103E60000BF04DEC0BF0230E0C6E02C10BF04DEC81
:103E70000BF0240E0C6E03C10BF04DEC0BF000C1E7
:103E800061F501C162F502C163F503C164F558EF44
:103E90001FF004014C0E826FABEC0EF00401490ED2
:103EA000826FABEC0EF004012C0E826FABEC0EF0C7
:103EB000250E64EC0BF0E8CF00F1260E64EC0BF05D
:103EC000E8CF01F1270E64EC0BF0E8CF02F1280EE9
:103ED00064EC0BF0E8CF03F14FEC31F012EC2FF073
:103EE0000401730E826FABEC0EF004012C0E826F96
:103EF000ABEC0EF0C6EC31F0290E64EC0BF0E8CF21
:103F000000F14FEC31F012EC2FF004016D0E826FD6
:103F1000ABEC0EF004012C0E826FABEC0EF05BC527
:103F200000F15CC501F15DC502F15EC503F14FEC26
:103F300031F012EC2FF00401730E826FABEC0EF037
:103F400004012C0E826FABEC0EF0C6EC31F060C5B4
:103F500000F14FEC31F012EC2FF004016D0E826F86
:103F6000ABEC0EF004012C0E826FABEC0EF061C5D1
:103F700000F162C501F163C502F164C503F1DBEC38
:103F80002AF004012C0E826FABEC0EF0B5EC0EF0B3
:103F9000C0EF2AF083C32AF184C32BF185C32CF12F
:103FA00086C32DF187C32EF188C32FF189C330F169
:103FB0008AC331F18BC332F18CC333F1010114ECAC
:103FC00032F08BEC31F0160E0C6E00C10BF04DECA4
:103FD0000BF0170E0C6E01C10BF04DEC0BF0180E30
:103FE0000C6E02C10BF04DEC0BF0190E0C6E03C100
:103FF0000BF04DEC0BF000C18EF101C18FF102C14D
:1040000090F103C191F100C192F101C193F102C19C
:1040100094F103C195F1ACEF20F083C32AF184C37E
:104020002BF185C32CF186C32DF187C32EF188C3F4
:104030002FF189C330F18AC331F18BC332F18CC3C4
:1040400033F1010114EC32F08BEC31F000C18EF150
:1040500001C18FF102C190F103C191F100C192F150
:1040600001C193F102C194F103C195F1ACEF20F0CD
:1040700083C32AF184C32BF185C32CF186C32DF1B0
:1040800087C32EF188C32FF189C330F18AC331F180
:104090008CC332F18DC333F1010114EC32F08BEC9F
:1040A00031F00101000E046F000E056F010E066F66
:1040B000000E076FC2EC30F01A0E0C6E00C10BF050
:1040C0004DEC0BF01B0E0C6E01C10BF04DEC0BF028
:1040D0001C0E0C6E02C10BF04DEC0BF01D0E0C6EA5
:1040E00003C10BF04DEC0BF000C196F101C197F14B
:1040F00002C198F103C199F1ACEF20F083C32AF11A
:1041000084C32BF185C32CF186C32DF187C32EF117
:1041100088C32FF189C330F18AC331F18CC332F1E6
:104120008DC333F1010114EC32F08BEC31F001015D
:10413000000E046F000E056F010E066F000E076F74
:10414000C2EC30F000C196F101C197F102C198F1C3
:1041500003C199F1ACEF20F0160E64EC0BF0E8CF40
:1041600000F1170E64EC0BF0E8CF01F1180E64ECCF
:104170000BF0E8CF02F1190E64EC0BF0E8CF03F17D
:104180004FEC31F012EC2FF00401730E826FABECA8
:104190000EF004012C0E826FABEC0EF08EC100F11C
:1041A0008FC101F190C102F191C103F14FEC31F0E7
:1041B00012EC2FF00401730E826FABEC0EF00401D1
:1041C0002C0E826FABEC0EF01A0E64EC0BF0E8CF05
:1041D00000F11B0E64EC0BF0E8CF01F11C0E64EC57
:1041E0000BF0E8CF02F11D0E64EC0BF0E8CF03F109
:1041F000DBEC2AF004012C0E826FABEC0EF096C1C2
:1042000000F197C101F198C102F199C103F1DBEC12
:104210002AF0B5EC0EF0C0EF2AF00401690E826FAF
:10422000ABEC0EF004012C0E826FABEC0EF0010132
:10423000040E006F000E016F000E026F000E036F80
:104240004FEC31F02CC182F40401300E8227ABEC2C
:104250000EF02DC182F40401300E8227ABEC0EF07B
:104260002EC182F40401300E8227ABEC0EF02FC178
:1042700082F40401300E8227ABEC0EF030C182F4E0
:104280000401300E8227ABEC0EF031C182F4040140
:10429000300E8227ABEC0EF032C182F40401300EF6
:1042A0008227ABEC0EF033C182F40401300E82277A
:1042B000ABEC0EF004012C0E826FABEC0EF00101A2
:1042C0000E0E006F000E016F000E026F000E036FE6
:1042D0004FEC31F02CC182F40401300E8227ABEC9C
:1042E0000EF02DC182F40401300E8227ABEC0EF0EB
:1042F0002EC182F40401300E8227ABEC0EF02FC1E8
:1043000082F40401300E8227ABEC0EF030C182F44F
:104310000401300E8227ABEC0EF031C182F40401AF
:10432000300E8227ABEC0EF032C182F40401300E65
:104330008227ABEC0EF033C182F40401300E8227E9
:10434000ABEC0EF004012C0E826FABEC0EF0010111
:10435000520E006F000E016F000E026F000E036F11
:104360004FEC31F02CC182F40401300E8227ABEC0B
:104370000EF02DC182F40401300E8227ABEC0EF05A
:104380002EC182F40401300E8227ABEC0EF02FC157
:1043900082F40401300E8227ABEC0EF030C182F4BF
:1043A0000401300E8227ABEC0EF031C182F404011F
:1043B000300E8227ABEC0EF032C182F40401300ED5
:1043C0008227ABEC0EF033C182F40401300E822759
:1043D000ABEC0EF004012C0E826FABEC0EF0200E55
:1043E000F86EF76AF66A04010900F5CF82F4ABECC7
:1043F0000EF00900F5CF82F4ABEC0EF00900F5CF1A
:1044000082F4ABEC0EF00900F5CF82F4ABEC0EF0C9
:104410000900F5CF82F4ABEC0EF00900F5CF82F481
:10442000ABEC0EF00900F5CF82F4ABEC0EF0090016
:10443000F5CF82F4ABEC0EF0B5EC0EF0C0EF2AF045
:104440008351630AD8A4BEEF2AF08451610AD8A42C
:10445000BEEF2AF085516C0AD8A4BEEF2AF086512F
:10446000410A3FE08651440A1BE08651420AD8B413
:1044700084EF22F08651350AD8B44AEF2CF08651E9
:10448000360AD8B49FEF2CF08651370AD8B408EF1B
:104490002DF08651380AD8B466EF2DF0BEEF2AF021
:1044A0000798079A04017A0E826FABEC0EF00401B4
:1044B000780E826FABEC0EF00401640E826FABECF1
:1044C0000EF00401550E826FABEC0EF06DEF22F092
:1044D00004014C0E826FABEC0EF0B5EC0EF0C0EFA9
:1044E0002AF00788079A04017A0E826FABEC0EF06F
:1044F0000401410E826FABEC0EF00401610E826F7D
:10450000ABEC0EF061EF22F00798078A04017A0EF7
:10451000826FABEC0EF00401420E826FABEC0EF03A
:104520000401610E826FABEC0EF061EF22F001012D
:104530006667A2EF22F06767A2EF22F06867A2EF3A
:1045400022F0696716D001014F67AEEF22F0506785
:10455000AEEF22F05167AEEF22F052670AD00101B0
:10456000000E006F000E016F000E026F000E036F51
:10457000120011B80AD00101620E046F010E056F1E
:10458000000E066F000E076F09D00101A70E046F21
:10459000020E056F000E066F000E076F66C100F178
:1045A00067C101F168C102F169C103F1B1EC30F0FA
:1045B00003BF4BEF23F0119A119C0101000E046F11
:1045C000A80E056F550E066F020E076F66C100F14B
:1045D00067C101F168C102F169C103F166C18AF1E5
:1045E00067C18BF168C18CF169C18DF1B1EC30F01C
:1045F00003BF0BD00101000E8A6FA80E8B6F550E02
:104600008C6F020E8D6F118A119C0E0E64EC0BF0F4
:10461000E8CF18F10F0E64EC0BF0E8CF19F1100E93
:1046200064EC0BF0E8CF1AF1110E64EC0BF0E8CF5C
:104630001BF1FAEC2FF08AC104F18BC105F18CC19A
:1046400006F18DC107F1B1EC30F00782BEEC2FF01E
:10465000FAEC2FF00792BEEC2FF08AC100F18BC16B
:1046600001F18CC102F18DC103F10792BEEC2FF074
:10467000CC0E046FE00E056F870E066F050E076FF8
:10468000B1EC30F000C118F101C119F102C11AF109
:1046900003C11BF140D013AA50EF23F0138E139ADD
:1046A000119C119A0101800E006F1A0E016F060E07
:1046B000026F000E036F4FC104F150C105F151C1EB
:1046C00006F152C107F1B1EC30F003AF05D0C6ECF2
:1046D00031F0118C119A12000E0E64EC0BF0E8CF41
:1046E00018F10F0E64EC0BF0E8CF19F1100E64EC2A
:1046F0000BF0E8CF1AF1110E64EC0BF0E8CF1BF1D0
:104700004FC100F150C101F151C102F152C103F199
:104710000782BEEC2FF018C100F119C101F11AC1D6
:1047200002F11BC103F112000784BAC166F1BBC1DB
:1047300067F1BCC168F1BDC169F14BC14FF14CC11A
:1047400050F14DC151F14EC152F157C159F158C10B
:104750005AF1079401016667B5EF23F06767B5EF7B
:1047600023F06867B5EF23F0696716D001014F6742
:10477000C1EF23F05067C1EF23F05167C1EF23F081
:1047800052670AD00101000E006F000E016F000E8B
:10479000026F000E036F120011B80AD00101620E01
:1047A000046F010E056F000E066F000E076F09D033
:1047B0000101A70E046F020E056F000E066F000EBA
:1047C000076F66C100F167C101F168C102F169C1FB
:1047D00003F1B1EC30F003BF4DEF24F00101000E06
:1047E000046FA80E056F550E066F020E076F66C1A7
:1047F00000F167C101F168C102F169C103F166C14D
:104800008AF167C18BF168C18CF169C18DF1B1EC9E
:1048100030F003BF09D00101000E8A6FA80E8B6F24
:10482000550E8C6F020E8D6FFAEC2FF000C104F163
:1048300001C105F102C106F103C107F1000E006FCD
:10484000A00E016F980E026F7B0E036FE2EC30F04A
:1048500000C118F101C119F102C11AF103C11BF124
:10486000000E006FA00E016F980E026F7B0E036F9B
:104870008AC104F18BC105F18CC106F18DC107F12C
:10488000E2EC30F018C104F119C105F11AC106F1CA
:104890001BC107F1B1EC30F012000101A80E006F4E
:1048A000610E016F000E026F000E036F4FC104F125
:1048B00050C105F151C106F152C107F1B1EC30F020
:1048C00003AF0AD00101A80E006F610E016F000E48
:1048D000026F000E036F00D0C80E006FAF0E016FA5
:1048E000000E026F000E036F4FC104F150C105F1BD
:1048F00051C106F152C107F1C2EC30F01200078439
:10490000BAC166F1BBC167F1BCC168F1BDC169F153
:104910004BC14FF14CC150F14DC151F14EC152F15B
:1049200057C159F158C15AF1079401016667A0EFC8
:1049300024F06767A0EF24F06867A0EF24F06967B0
:1049400016D001014F67ACEF24F05067ACEF24F0B4
:104950005167ACEF24F052670AD00101000E006FDE
:10496000000E016F000E026F000E036F120011B8EF
:104970000AD00101620E046F010E056F000E066F72
:10498000000E076F09D00101A70E046F020E056F1C
:10499000000E066F000E076F66C100F167C101F1DE
:1049A00068C102F169C103F1B1EC30F003BF62EFFD
:1049B00025F00101000E046FA80E056F550E066F5D
:1049C000020E076F66C100F167C101F168C102F113
:1049D00069C103F166C18AF167C18BF168C18CF1CD
:1049E00069C18DF1B1EC30F003BF09D00101000EB7
:1049F0008A6FA80E8B6F550E8C6F020E8D6F010E95
:104A0000006F000E016F000E026F000E036F8AC16F
:104A100004F18BC105F18CC106F18DC107F1E2EC07
:104A200030F018C104F119C105F11AC106F11BC11A
:104A300007F14FEC31F02AC182F40401300E8227D5
:104A4000ABEC0EF02BC182F40401300E8227ABECEC
:104A50000EF02CC182F40401300E8227ABEC0EF074
:104A60002DC182F40401300E8227ABEC0EF02EC172
:104A700082F40401300E8227ABEC0EF02FC182F4D9
:104A80000401300E8227ABEC0EF030C182F4040139
:104A9000300E8227ABEC0EF031C182F40401300EEF
:104AA0008227ABEC0EF032C182F40401300E822773
:104AB000ABEC0EF033C182F40401300E8227ABEC74
:104AC0000EF012004FC100F150C101F151C102F1CD
:104AD00052C103F101014FEC31F012EC2FF0120042
:104AE0000401730E826FABEC0EF004012C0E826F8A
:104AF000ABEC0EF0078462C166F163C167F164C17B
:104B000068F165C169F14BC14FF14CC150F14DC124
:104B100051F14EC152F157C159F158C15AF10794A0
:104B200096EC25F0B5EC0EF0C0EF2AF066C100F16E
:104B300067C101F168C102F169C103F101014FECE4
:104B400031F012EC2FF00401630E826FABEC0EF02B
:104B500004012C0E826FABEC0EF04FC100F150C17E
:104B600001F151C102F152C103F101014FEC31F0E9
:104B700012EC2FF00401660E826FABEC0EF0040114
:104B80002C0E826FABEC0EF0C6EC31F059C100F187
:104B90005AC101F101014FEC31F012EC2FF0040188
:104BA000740E826FABEC0EF0120010820401530EF3
:104BB000826FABEC0EF004012C0E826FABEC0EF0AA
:104BC00083C32AF184C32BF185C32CF186C32DF155
:104BD00087C32EF188C32FF189C330F18AC331F125
:104BE0008BC332F18CC333F1010114EC32F08BEC46
:104BF00031F000C166F101C167F102C168F103C182
:104C000069F18EC32AF18FC32BF190C32CF191C3AC
:104C10002DF192C32EF193C32FF194C330F195C3BC
:104C200031F196C332F197C333F1010114EC32F044
:104C30008BEC31F000C14FF101C150F102C151F1D3
:104C400003C152F107EC32F099C32FF19AC330F14E
:104C50009BC331F19CC332F19DC333F1010114ECCC
:104C600032F08BEC31F000C159F101C15AF196ECF0
:104C700025F004012C0E826FABEC0EF050EF26F005
:104C8000118E1CA002D01CAE108C1BBE02D01BA427
:104C9000108E03018251520A02E10F8201D00F925D
:104CA0008251750A02E1108401D010948251550A94
:104CB00002E1108601D010968351310A03E113827C
:104CC000138402D01392139403018351660A01E006
:104CD00056D00401660E826FABEC0EF004012C0E70
:104CE000826FABEC0EF094EC23F04FEC31F02AC164
:104CF00082F40401300E8227ABEC0EF02BC182F45B
:104D00000401300E8227ABEC0EF02CC182F40401BA
:104D1000300E8227ABEC0EF02DC182F40401300E70
:104D20008227ABEC0EF02EC182F40401300E8227F4
:104D3000ABEC0EF02FC182F40401300E8227ABECF5
:104D40000EF030C182F40401300E8227ABEC0EF07D
:104D500031C182F40401300E8227ABEC0EF032C177
:104D600082F40401300E8227ABEC0EF033C182F4E2
:104D70000401300E8227ABEC0EF0BEEF2AF011A03A
:104D800003D011A401D01084078410B229EF27F0BA
:104D900010A40DEF27F0BAC166F1BBC167F1BCC129
:104DA00068F1BDC169F1BEC16AF1BFC16BF1C0C19B
:104DB0006CF1C1C16DF1C2C16EF1C3C16FF1C4C16B
:104DC00070F1C5C171F1C6C172F1C7C173F1C8C13B
:104DD00074F1C9C175F1CAC176F1CBC177F1CCC10B
:104DE00078F1CDC179F1CEC17AF1CFC17BF1D0C1DB
:104DF0007CF1D1C17DF1D2C17EF1D3C17FF1D4C1AB
:104E000080F1D5C181F1D6C182F1D7C183F1D8C17A
:104E100084F1D9C185F115EF27F062C166F163C154
:104E200067F164C168F165C169F1BAC186F1BBC1BE
:104E300087F1BCC188F1BDC189F14BC14FF14CC1B3
:104E400050F14DC151F14EC152F157C159F158C104
:104E50005AF107940FA04BEF27F00101966738EF46
:104E600027F0976738EF27F0986738EF27F09967B2
:104E70003CEF27F04BEF27F097EC22F096C104F1BE
:104E800097C105F198C106F199C107F1B1EC30F075
:104E900003BF84EF2AF097EC22F00101000E046FAB
:104EA000000E056F010E066F000E076FE2EC30F08A
:104EB00011A02AD011A228D04FEC31F0296701D0DF
:104EC00005D004012D0E826FABEC0EF030C182F4E0
:104ED0000401300E8227ABEC0EF031C182F40401E4
:104EE000300E8227ABEC0EF032C182F40401300E9A
:104EF0008227ABEC0EF033C182F40401300E82271E
:104F0000ABEC0EF0B5EC0EF012A8C5D012981DC097
:104F10001EF01E3A1E42070E1E1600011E50000A09
:104F2000D8B417EF28F000011E50010AD8B4A3EF3F
:104F300027F000011E50020AD8B4A1EF27F049EF74
:104F400028F049EF28F0C6EC31F02EC001F12FC057
:104F500000F1D89001330033D890013300330101C0
:104F6000630E046F000E056F000E066F000E076FD4
:104F7000E2EC30F0280E046F000E056F000E066F95
:104F8000000E076FB1EC30F000C131F0C6EC31F02B
:104F90002CC001F1019F019D2DC000F10101A40E63
:104FA000046F000E056F000E066F000E076FE2EC37
:104FB00030F000C130F000C104F101C105F102C1BF
:104FC00006F103C107F1640E006F000E016F000EC1
:104FD000026F000E036FB1EC30F0050E046F000E8F
:104FE000056F000E066F000E076FE2EC30F000C197
:104FF00004F101C105F102C106F103C107F1C6ECDC
:1050000031F031C000F1B1EC30F000C132F032C00B
:10501000E8FF050F315C03E78A8449EF28F032C0CE
:10502000E8FF0A0F315C01E68A9449EF28F000C1DD
:1050300024F101C125F102C126F103C127F1C6EC1B
:1050400031F0CCEC31F01D501F0BE8CF00F1010125
:10505000640E046F000E056F000E066F000E076FE2
:10506000C2EC30F024C104F125C105F126C106F1DE
:1050700027C107F1B1EC30F003BF02D08A9401D010
:105080008A8424C100F125C101F126C102F127C1A2
:1050900003F1C0EF2AF000C124F101C125F102C1E2
:1050A00026F103C127F110AE4DD0109E00C108F1CA
:1050B00001C109F102C10AF103C10BF14FEC31F05A
:1050C00030C1E2F131C1E3F132C1E4F133C1E5F1C4
:1050D00008C100F109C101F10AC102F10BC103F1DC
:1050E00001016C0E046F070E056F000E066F000EB7
:1050F000076FB1EC30F003BF04D00101550EE66F2D
:105100001CD008C100F109C101F10AC102F10BC1B3
:1051100003F10101A40E046F060E056F000E066F69
:10512000000E076FB1EC30F003BF04D001017F0E19
:10513000E66F03D00101FF0EE66F1F8E11AE84EF04
:105140002AF0119E24C100F125C101F126C102F10E
:1051500027C103F111A005D011A203D00FB084EF35
:105160002AF010A4BBEF28F00401750E826FABEC9F
:105170000EF0C0EF28F00401720E826FABEC0EF05F
:1051800004012C0E826FABEC0EF04FEC31F029676E
:10519000CFEF28F00401200E826FD2EF28F0040137
:1051A0002D0E826FABEC0EF030C182F40401300E94
:1051B0008227ABEC0EF031C182F40401300E82275D
:1051C000ABEC0EF004012E0E826FABEC0EF032C190
:1051D00082F40401300E8227ABEC0EF033C182F46E
:1051E0000401300E8227ABEC0EF004016D0E826FCD
:1051F000ABEC0EF004012C0E826FABEC0EF04FC145
:1052000000F150C101F151C102F152C103F101019C
:105210004FEC31F012EC2FF00401480E826FABEC32
:105220000EF004017A0E826FABEC0EF004012C0E2E
:10523000826FABEC0EF066C100F167C101F168C18D
:1052400002F169C103F101014FEC31F012EC2FF0D2
:105250000401630E826FABEC0EF004012C0E826F22
:10526000ABEC0EF066C100F167C101F168C102F15B
:1052700069C103F101010A0E046F000E056F000EF3
:10528000066F000E076FC2EC30F0000E046F120EB6
:10529000056F000E066F000E076FE2EC30F04FEC6A
:1052A00031F02AC182F40401300E8227ABEC0EF0FB
:1052B0002BC182F40401300E8227ABEC0EF02CC11E
:1052C00082F40401300E8227ABEC0EF02DC182F483
:1052D0000401300E8227ABEC0EF02EC182F40401E3
:1052E000300E8227ABEC0EF02FC182F40401300E99
:1052F0008227ABEC0EF030C182F40401300E82271D
:10530000ABEC0EF004012E0E826FABEC0EF031C14F
:1053100082F40401300E8227ABEC0EF032C182F42D
:105320000401300E8227ABEC0EF033C182F404018D
:10533000300E8227ABEC0EF00401730E826FABECE3
:105340000EF004012C0E826FABEC0EF0C6EC31F0C7
:1053500059C100F15AC101F1EAEC2BF013A200EFA0
:105360002AF004012C0E826FABEC0EF086C166F1C0
:1053700087C167F188C168F189C169F197EC22F0B2
:105380000101000E046F000E056F010E066F000E86
:10539000076FE2EC30F04FEC31F02967D5EF29F0E0
:1053A0000401200E826FD8EF29F004012D0E826FC8
:1053B000ABEC0EF030C182F40401300E8227ABEC6E
:1053C0000EF031C182F40401300E8227ABEC0EF0F6
:1053D00004012E0E826FABEC0EF032C182F4040198
:1053E000300E8227ABEC0EF033C182F40401300E94
:1053F0008227ABEC0EF004016D0E826FABEC0EF069
:1054000003018351460A01E007D004012C0E826F8C
:10541000ABEC0EF07FEC24F013A433EF2AF0040180
:105420002C0E826FABEC0EF013AC21EF2AF00401CE
:10543000500E826FABEC0EF0139C1398139A33EF5F
:105440002AF013AE2EEF2AF00401460E826FABEC69
:105450000EF0139E1398139A33EF2AF00401530EA3
:10546000826FABEC0EF038B04AEF2AF004012C0E3C
:10547000826FABEC0EF08BB045EF2AF00401440EC6
:10548000826FABEC0EF04AEF2AF00401530E826FEC
:10549000ABEC0EF00FB250EF2AF00FA082EF2AF023
:1054A00004012C0E826FABEC0EF0200EF86EF76A42
:1054B000F66A04010900F5CF82F4ABEC0EF00900A6
:1054C000F5CF82F4ABEC0EF00900F5CF82F4ABEC33
:1054D0000EF00900F5CF82F4ABEC0EF00900F5CF29
:1054E00082F4ABEC0EF00900F5CF82F4ABEC0EF0D9
:1054F0000900F5CF82F4ABEC0EF00900F5CF82F491
:10550000ABEC0EF0B5EC0EF00F90109E1298C0EFC1
:105510002AF00401630E826FABEC0EF004012C0E36
:10552000826FABEC0EF0C6EC2AF004012C0E826FF9
:10553000ABEC0EF039EC2BF004012C0E826FABECCF
:105540000EF0B5EC2BF004012C0E826FABEC0EF0DC
:105550000101F80E006FCD0E016F660E026F030E93
:10556000036FDBEC2AF004012C0E826FABEC0EF023
:10557000CBEC2BF0B5EC0EF0C0EF2AF0B5EC0EF052
:105580000301C26B07901092CFEF2DF0D8900E0E52
:1055900064EC0BF0E8CF00F10F0E64EC0BF0E8CFF9
:1055A00001F1100E64EC0BF0E8CF02F1110E64EC87
:1055B0000BF0E8CF03F10101000E046F000E056F40
:1055C000010E066F000E076FE2EC30F04FEC31F089
:1055D0002AC182F40401300E8227ABEC0EF02BC1FD
:1055E00082F40401300E8227ABEC0EF02CC182F461
:1055F0000401300E8227ABEC0EF02DC182F40401C1
:10560000300E8227ABEC0EF02EC182F40401300E76
:105610008227ABEC0EF02FC182F40401300E8227FA
:10562000ABEC0EF030C182F40401300E8227ABECFB
:105630000EF031C182F40401300E8227ABEC0EF083
:1056400004012E0E826FABEC0EF032C182F4040125
:10565000300E8227ABEC0EF033C182F40401300E21
:105660008227ABEC0EF004016D0E826FABEC0EF0F6
:105670001200120E64EC0BF0E8CF00F1130E64EC94
:105680000BF0E8CF01F1140E64EC0BF0E8CF02F15F
:10569000150E64EC0BF0E8CF03F101010A0E046F64
:1056A000000E056F000E066F000E076FC2EC30F0A3
:1056B000000E046F120E056F000E066F000E076FCE
:1056C000E2EC30F04FEC31F02AC182F40401300EEC
:1056D0008227ABEC0EF02BC182F40401300E82273E
:1056E000ABEC0EF02CC182F40401300E8227ABEC3F
:1056F0000EF02DC182F40401300E8227ABEC0EF0C7
:105700002EC182F40401300E8227ABEC0EF02FC1C3
:1057100082F40401300E8227ABEC0EF030C182F42B
:105720000401300E8227ABEC0EF004012E0E826FC6
:10573000ABEC0EF031C182F40401300E8227ABECE9
:105740000EF032C182F40401300E8227ABEC0EF071
:1057500033C182F40401300E8227ABEC0EF0040159
:10576000730E826FABEC0EF012000A0E64EC0BF0BD
:10577000E8CF00F10B0E64EC0BF0E8CF01F10C0E5A
:1057800064EC0BF0E8CF02F10D0E64EC0BF0E8CF07
:1057900003F1EAEF2BF0060E64EC0BF0E8CF00F11A
:1057A000070E64EC0BF0E8CF01F1080E64EC0BF08F
:1057B000E8CF02F1090E64EC0BF0E8CF03F1EAEF59
:1057C0002BF00101C6EC31F0078457C100F158C13C
:1057D00001F107940101E80E046F800E056F000EC1
:1057E000066F000E076FC2EC30F0000E046F040E5F
:1057F000056F000E066F000E076FE2EC30F0880EAA
:10580000046F130E056F000E066F000E076FB1ECEC
:1058100030F00A0E046F000E056F000E066F000ECA
:10582000076FE2EC30F04FEC31F0010129671EEF19
:105830002CF00401200E826F21EF2CF004012D0EBC
:10584000826FABEC0EF030C182F40401300E82277F
:10585000ABEC0EF031C182F40401300E8227ABECC8
:105860000EF032C182F40401300E8227ABEC0EF050
:1058700004012E0E826FABEC0EF033C182F40401F2
:10588000300E8227ABEC0EF00401430E826FABECBE
:105890000EF0120087C32AF188C32BF189C32CF1C3
:1058A0008AC32DF18BC32EF18CC32FF18DC330F140
:1058B0008EC331F190C332F191C333F10101296BF1
:1058C00014EC32F08BEC31F00101000E046F000E8D
:1058D000056F010E066F000E076FC2EC30F00E0E62
:1058E0000C6E00C10BF04DEC0BF00F0E0C6E01C1F5
:1058F0000BF04DEC0BF0100E0C6E02C10BF04DECEA
:105900000BF0110E0C6E03C10BF04DEC0BF004010B
:105910007A0E826FABEC0EF004012C0E826FABECB2
:105920000EF00401350E826FABEC0EF004012C0E6C
:10593000826FABEC0EF0C6EC2AF06DEF22F087C35D
:105940002AF188C32BF189C32CF18AC32DF18BC3B3
:105950002EF18CC32FF18DC330F18EC331F190C382
:1059600032F191C333F10101296B14EC32F08BEC6D
:1059700031F0880E046F130E056F000E066F000ED7
:10598000076FB6EC30F0000E046F040E056F000ECA
:10599000066F000E076FC2EC30F00101E80E046FD5
:1059A000800E056F000E066F000E076FE2EC30F000
:1059B0000A0E0C6E00C10BF04DEC0BF00B0E0C6ED2
:1059C00001C10BF04DEC0BF00C0E0C6E02C10BF094
:1059D0004DEC0BF00D0E0C6E03C10BF04DEC0BF00B
:1059E00004017A0E826FABEC0EF004012C0E826F74
:1059F000ABEC0EF00401360E826FABEC0EF004013E
:105A00002C0E826FABEC0EF0B5EC2BF06DEF22F0AC
:105A100087C32AF188C32BF189C32CF18AC32DF1E6
:105A20008BC32EF18CC32FF18DC330F18FC331F1B5
:105A300090C332F191C333F1010114EC32F08BECDD
:105A400031F0000E046F120E056F000E066F000E8F
:105A5000076FC2EC30F001010A0E046F000E056FF3
:105A6000000E066F000E076FE2EC30F0120E0C6EA7
:105A700000C10BF04DEC0BF0130E0C6E01C10BF0DE
:105A80004DEC0BF0140E0C6E02C10BF04DEC0BF054
:105A9000150E0C6E03C10BF04DEC0BF004017A0EE9
:105AA000826FABEC0EF004012C0E826FABEC0EF0AB
:105AB0000401370E826FABEC0EF004012C0E826FE6
:105AC000ABEC0EF039EC2BF06DEF22F087C32AF12E
:105AD00088C32BF189C32CF18AC32DF18BC32EF11E
:105AE0008CC32FF18DC330F18EC331F190C332F1ED
:105AF00091C333F10101296B14EC32F08BEC31F0DE
:105B0000880E046F130E056F000E066F000E076FF0
:105B1000B6EC30F0000E046F040E056F000E066F39
:105B2000000E076FC2EC30F00101E80E046F800E2A
:105B3000056F000E066F000E076FE2EC30F0060EE8
:105B40000C6E00C10BF04DEC0BF0070E0C6E01C19A
:105B50000BF04DEC0BF0080E0C6E02C10BF04DEC8F
:105B60000BF0090E0C6E03C10BF04DEC0BF00401B1
:105B70007A0E826FABEC0EF004012C0E826FABEC50
:105B80000EF00401380E826FABEC0EF004012C0E07
:105B9000826FABEC0EF0CBEC2BF06DEF22F007A890
:105BA00042EF2EF00101800E006F1A0E016F060EFB
:105BB000026F000E036F4BC104F14CC105F14DC1E2
:105BC00006F14EC107F1B1EC30F003BF88EF2EF0C3
:105BD0000CEC2FF04BC100F14CC101F14DC102F1B1
:105BE0004EC103F10782BEEC2FF018C104F119C1B8
:105BF00005F11AC106F11BC107F1F80E006FCD0EB9
:105C0000016F660E026F030E036FB1EC30F00E0EE3
:105C10000C6E00C10BF04DEC0BF00F0E0C6E01C1C1
:105C20000BF04DEC0BF0100E0C6E02C10BF04DECB6
:105C30000BF0110E0C6E03C10BF04DEC0BF0078452
:105C40000101C6EC31F057C100F158C101F10794D0
:105C50000A0E0C6E00C10BF04DEC0BF00B0E0C6E2F
:105C600001C10BF04DEC0BF00C0E0C6E02C10BF0F1
:105C70004DEC0BF00D0E0C6E03C10BF04DEC0BF068
:105C800088EF2EF007AA88EF2EF007840101C6ECFA
:105C900031F057C100F158C101F10794060E0C6EA6
:105CA00000C10BF04DEC0BF0070E0C6E01C10BF0B8
:105CB0004DEC0BF0080E0C6E02C10BF04DEC0BF02E
:105CC000090E0C6E03C10BF04DEC0BF0078462C1A2
:105CD00000F163C101F164C102F165C103F10794F0
:105CE000120E0C6E00C10BF04DEC0BF0130E0C6E8F
:105CF00001C10BF04DEC0BF0140E0C6E02C10BF059
:105D00004DEC0BF0150E0C6E03C10BF04DEC0BF0CF
:105D10000798079A0401805181197F0B0DE09EA816
:105D2000FED714EE00F081517F0BE126E750812B66
:105D30000F01AD6E8AEF2EF005012F51000AD8B485
:105D4000CBEF2EF081BAB0EF2EF015B2CBEF2EF0E4
:105D500005012F51010AD8B4C9EF2EF0C2EF2EF081
:105D600005012F51000AD8B4BFEF39F005012F51BA
:105D7000010AD8B4C9EF2EF000011650050AD8B4B4
:105D8000BFEF39F081B8CBEF2EF041EC33F0E7EC08
:105D900033F056EC39F081A4D2EF2EF09492949C1B
:105DA000D4EF2EF09482948CD9EF0DF018C100F14D
:105DB00019C101F11AC102F11BC103F1000E046FF8
:105DC000000E056F010E066F000E076FE2EC30F05B
:105DD00029A101EF2FF02051D8B401EF2FF018C105
:105DE00000F119C101F11AC102F11BC103F1000E4A
:105DF000046F000E056F0A0E066F000E076FE2ECCF
:105E000030F0120001010451001305510113065135
:105E100002130751031312000101186B196B1A6B5F
:105E20001B6B12002AC182F40401300E8227ABECF6
:105E30000EF02BC182F40401300E8227ABEC0EF081
:105E40002CC182F40401300E8227ABEC0EF02DC180
:105E500082F40401300E8227ABEC0EF02EC182F4E6
:105E60000401300E8227ABEC0EF02FC182F4040146
:105E7000300E8227ABEC0EF030C182F40401300EFC
:105E80008227ABEC0EF031C182F40401300E822780
:105E9000ABEC0EF032C182F40401300E8227ABEC81
:105EA0000EF033C182F40401300E8227ABEC0EF009
:105EB00012002FC182F40401300E8227ABEC0EF0E9
:105EC00030C182F40401300E8227ABEC0EF031C1F8
:105ED00082F40401300E8227ABEC0EF032C182F462
:105EE0000401300E8227ABEC0EF033C182F40401C2
:105EF000300E8227ABEC0EF01200060E216E060E5D
:105F0000226E060E236E212E83EF2FF0222E83EFBA
:105F10002FF0232E83EF2FF08B84020E216E020EC2
:105F2000226E020E236E212E93EF2FF0222E93EF7E
:105F30002FF0232E93EF2FF08B941200FF0E226E82
:105F400022C023F0030E216E8B84212EA4EF2FF0AC
:105F5000030E216E232EA4EF2FF08B9422C023F08A
:105F6000030E216E212EB2EF2FF0030E216E233E81
:105F7000B2EF2FF0222EA0EF2FF0120001010053FC
:105F800005E1015303E1025301E1002B81EC30F004
:105F9000C6EC31F03951006F3A51016F420E046F77
:105FA0004B0E056F000E066F000E076FC2EC30F04F
:105FB00000C104F101C105F102C106F103C107F1FD
:105FC00018C100F119C101F11AC102F11BC103F19D
:105FD00007B2EFEF2FF0B6EC30F0F1EF2FF0B1ECAD
:105FE00030F000C118F101C119F102C11AF103C169
:105FF0001BF11200C6EC31F059C100F15AC101F198
:10600000060E64EC0BF0E8CF04F1070E64EC0BF025
:10601000E8CF05F1080E64EC0BF0E8CF06F1090EAD
:1060200064EC0BF0E8CF07F1B1EC30F000C124F1E3
:1060300001C125F102C126F103C127F1290E046F28
:10604000000E056F000E066F000E076FC2EC30F0F9
:10605000EE0E046F430E056F000E066F000E076F05
:10606000B6EC30F024C104F125C105F126C106F1DA
:1060700027C107F1C2EC30F000C11CF101C11DF1D4
:1060800002C11EF103C11FF1120E64EC0BF0E8CF48
:1060900004F1130E64EC0BF0E8CF05F1140E64EC80
:1060A0000BF0E8CF06F1150E64EC0BF0E8CF07F12A
:1060B0000D0E006F000E016F000E026F000E036FD9
:1060C000C2EC30F0180E046F000E056F000E066F64
:1060D000000E076FE2EC30F01CC104F11DC105F1A8
:1060E0001EC106F11FC107F1B6EC30F06A0E046F55
:1060F0002A0E056F000E066F000E076FB1EC30F030
:106100001200BF0EFA6E200E3A6F396BD89000372E
:10611000013702370337D8B092EF30F03A2F87EFCC
:1061200030F039073A070353D8B412000331070B94
:1061300080093F6F03390F0B010F396F80EC5FF05F
:10614000406F390580EC5FF0405D405F396B3F3355
:10615000D8B0392739333FA9A7EF30F0405139275C
:1061600012000101EBEC31F0D8B012000101035133
:106170000719346FAEEC31F0D8900751031934AFE2
:10618000800F12000101346BD2EC31F0D8A0E8ECA2
:1061900031F0D8B01200BDEC31F0C6EC31F01F0E7A
:1061A000366FFEEC31F00B35D8B0AEEC31F0D8A044
:1061B0000335D8B01200362FD1EF30F034B1D5EC22
:1061C00031F012000101346B045105110611071161
:1061D0000008D8A0D2EC31F0D8A0E8EC31F0D8B06B
:1061E0001200086B096B0A6B0B6BFEEC31F01F0E93
:1061F000366FFEEC31F007510B5DD8A40CEF31F097
:1062000006510A5DD8A40CEF31F00551095DD8A400
:106210000CEF31F00451085DD8A01FEF31F00451AC
:10622000085F0551D8A0053D095F0651D8A0063D7D
:106230000A5F0751D8A0073D0B5FD8900081362F29
:10624000F9EF30F034B1D5EC31F0346BD2EC31F001
:10625000D89002EC32F007510B5DD8A43CEF31F03E
:1062600006510A5DD8A43CEF31F00551095DD8A470
:106270003CEF31F00451085DD8A04BEF31F0003F06
:106280004BEF31F0013F4BEF31F0023F4BEF31F07C
:10629000032BD8B4120034B1D5EC31F01200010157
:1062A000346BD2EC31F0D8B0120007EC32F0200E93
:1062B000366F003701370237033711EE33F00A0E1D
:1062C000376FE7360A0EE75CD8B0E76EE552372F36
:1062D00061EF31F0362F59EF31F034B12981D89088
:1062E000120007EC32F0200E366F0037013702370C
:1062F000033711EE33F00A0E376FE7360A0EE75C0C
:10630000D8B0E76EE552372F7DEF31F0362F75EFBD
:1063100031F0D890120001010A0E346F200E366F52
:1063200011EE29F03451376F0A0ED890E652D8B0EA
:10633000E726E732372F96EF31F00333023301338C
:106340000033362F90EF31F0E750FF0FD8A0033520
:10635000D8B0120029B1D5EC31F012000451002759
:106360000551D8B0053D01270651D8B0063D02279A
:106370000751D8B0073D032712000051086F0151A3
:10638000096F02510A6F03510B6F12000101006B7C
:10639000016B026B036B12000101046B056B066B52
:1063A000076B12000335D8A012000351800B001FA9
:1063B000011F021F031F003FE5EF31F0013FE5EF32
:1063C00031F0023FE5EF31F0032B342B03251200AF
:1063D0000735D8A012000751800B041F051F061FA8
:1063E000071F043FFBEF31F0053FFBEF31F0063FA5
:1063F000FBEF31F0072B342B072512000037013754
:1064000002370337083709370A370B371200010103
:10641000296B2A6B2B6B2C6B2D6B2E6B2F6B306BC0
:10642000316B326B336B120001012A510F0B2A6F53
:106430002B510F0B2B6F2C510F0B2C6F2D510F0B62
:106440002D6F2E510F0B2E6F2F510F0B2F6F3051C1
:106450000F0B306F31510F0B316F32510F0B326F09
:1064600033510F0B336F120000C124F101C125F12C
:1064700002C126F103C127F104C100F105C101F1F8
:1064800006C102F107C103F124C104F125C105F1E0
:1064900026C106F127C107F1120000012550FE0AAE
:1064A000D8B45BEF32F000012550FD0AD8B45BEFA1
:1064B00032F0898401D08994000EC76E220EC66E18
:1064C000050EE82EFED7120000012550FE0AD8B4B2
:1064D00072EF32F000012550FD0AD8B472EF32F0AD
:1064E000899401D08984050EE82EFED712004DEC68
:1064F00032F000012550FD0AD8B48AEF32F09E96A2
:10650000C69E000EC96EFF0E9EB602D0E82EFCD7C6
:1065100093EF32F09E96C69E010EC96EFF0E9EB698
:1065200002D0E82EFCD79E96C69E000EC96EFF0EC6
:106530009EB602D0E82EFCD7C9CFAFF59E96C69E78
:10654000000EC96EFF0E9EB602D0E82EFCD7C9CF52
:10655000B0F59E96C69E000EC96EFF0E9EB602D086
:10656000E82EFCD7C9CFB1F59E96C69E000EC96E27
:10657000FF0E9EB602D0E82EFCD7C9CFB2F59E968C
:10658000C69E000EC96EFF0E9EB602D0E82EFCD746
:10659000C9CFB3F59E96C69E000EC96EFF0E9EB67D
:1065A00002D0E82EFCD7C9CFB4F59E96C69E000E49
:1065B000C96EFF0E9EB602D0E82EFCD7C9CFB5F546
:1065C00064EC32F012004DEC32F000012550FD0A6F
:1065D000D8B4F6EF32F09E96C69E800EC96EFF0EBE
:1065E0009EB602D0E82EFCD7FFEF32F09E96C69EF4
:1065F000810EC96EFF0E9EB602D0E82EFCD79E9685
:10660000C69EAFC5C9FFFF0E9EB602D0E82EFCD7CE
:106610009E96C69EB0C5C9FFFF0E9EB602D0E82E5C
:10662000FCD79E96C69EB1C5C9FFFF0E9EB602D08E
:10663000E82EFCD79E96C69EB2C5C9FFFF0E9EB639
:1066400002D0E82EFCD79E96C69EB3C5C9FFFF0EAA
:106650009EB602D0E82EFCD79E96C69EB4C5C9FF52
:10666000FF0E9EB602D0E82EFCD79E96C69EB5C5FC
:10667000C9FFFF0E9EB602D0E82EFCD764EC32F0C4
:1066800012004DEC32F000012550FD0AD8B454EF51
:1066900033F09E96C69E070EC96EFF0E9EB602D0C0
:1066A000E82EFCD75DEF33F09E96C69E090EC96EAC
:1066B000FF0E9EB602D0E82EFCD79E96C69E000E18
:1066C000C96EFF0E9EB602D0E82EFCD7C9CFAFF53B
:1066D0009E96C69E000EC96EFF0E9EB602D0E82E94
:1066E000FCD7C9CFB0F59E96C69E000EC96EFF0EB0
:1066F0009EB602D0E82EFCD7C9CFB1F59E96C69EB5
:10670000000EC96EFF0E9EB602D0E82EFCD7C9CF90
:10671000B2F564EC32F04DEC32F09E96C69E26C087
:10672000C9FFFF0E9EB602D0E82EFCD79E96C69EED
:10673000000EC96EFF0E9EB602D0E82EFCD7C9CF60
:10674000B6F564EC32F012004DEC32F00001255049
:10675000FD0AD8B4B7EF33F09E96C69E870EC96E79
:10676000FF0E9EB602D0E82EFCD7C0EF33F09E9607
:10677000C69E890EC96EFF0E9EB602D0E82EFCD7CB
:106780009E96C69E000EC96EFF0E9EB602D0E82EE3
:10679000FCD79E96C69E800EC96EFF0E9EB602D096
:1067A000E82EFCD79E96C69E800EC96EFF0E9EB642
:1067B00002D0E82EFCD79E96C69E800EC96EFF0EB4
:1067C0009EB602D0E82EFCD764EC32F01200000135
:1067D0002550FE0AD8B4F6EF33F000012550FD0A2B
:1067E000D8B40DEF34F041EC33F012004DEC32F040
:1067F0009E96C69E8F0EC96EFF0E9EB602D0E82EE4
:10680000FCD79E96C69E000EC96EFF0E9EB602D0A5
:10681000E82EFCD764EC32F012004DEC32F09E967C
:10682000C69E8E0EC96EFF0E9EB602D0E82EFCD715
:106830009E96C69E000EC96EFF0E9EB602D0E82E32
:10684000FCD764EC32F0120000012550FE0AD8B4E7
:106850005DEF34F000012550FD0AD8B48AEF34F022
:106860004DEC32F09E96C69E27C0C9FFFF0E9EB625
:1068700002D0E82EFCD79E96C69E010EC96EFF0E72
:106880009EB602D0E82EFCD764EC32F04DEC32F02C
:106890009E96C69E910EC96EFF0E9EB602D0E82E41
:1068A000FCD79E96C69EA50EC96EFF0E9EB602D060
:1068B000E82EFCD764EC32F012004DEC32F09E96DC
:1068C000C69E27C0C9FFFF0E9EB602D0E82EFCD799
:1068D0009E96C69E450EC96EFF0E9EB602D0E82E4D
:1068E000FCD764EC32F04DEC32F09E96C69E8F0ED3
:1068F000C96EFF0E9EB602D0E82EFCD79E96C69EAD
:10690000000EC96EFF0E9EB602D0E82EFCD764ECD6
:1069100032F012004DEC32F09E96C69E27C0C9FFA1
:10692000FF0E9EB602D0E82EFCD79E96C69E3D0E68
:10693000C96EFF0E9EB602D0E82EFCD764EC32F092
:106940004DEC32F09E96C69E8F0EC96EFF0E9EB61F
:1069500002D0E82EFCD79E96C69EA90EC96EFF0EE9
:106960009EB602D0E82EFCD764EC32F012004DEC5B
:1069700032F09E96C69E27C0C9FFFF0E9EB602D07B
:10698000E82EFCD79E96C69E810EC96EFF0E9EB65F
:1069900002D0E82EFCD764EC32F012004DEC32F05D
:1069A0009E96C69E27C0C9FFFF0E9EB602D0E82E57
:1069B000FCD79E96C69E010EC96EFF0E9EB602D0F3
:1069C000E82EFCD764EC32F012004DEC32F09E96CB
:1069D000C69E910EC96EFF0E9EB602D0E82EFCD761
:1069E0009E96C69EA50EC96EFF0E9EB602D0E82EDC
:1069F000FCD764EC32F012004DEC32F09E96C69E4D
:106A0000910EC96EFF0E9EB602D0E82EFCD79E9660
:106A1000C69E000EC96EFF0E9EB602D0E82EFCD7B1
:106A200064EC32F012000501256B266B276B286B96
:106A3000899A400EC76E200EC66E9E96C69E030EA5
:106A4000C96EFF0E9EB602D0E82EFCD79E96C69E5B
:106A500027C5C9FFFF0E9EB602D0E82EFCD79E9632
:106A6000C69E26C5C9FFFF0E9EB602D0E82EFCD7F3
:106A70009E96C69E25C5C9FFFF0E9EB602D0E82E83
:106A8000FCD79E96C69EC952FF0E9EB602D0E82E37
:106A9000FCD7898A0F01C950FF0A01E112000501E4
:106AA0002E51130A05E005012E51170A0CE01200C1
:106AB0000501E00E256FFF0E266F0F0E276F000EEB
:106AC000286F6CEF35F00501E00E256FFF0E266F85
:106AD000FF0E276F000E286F899A400EC76E200E9A
:106AE000C66E9E96C69E030EC96EFF0E9EB602D05F
:106AF000E82EFCD79E96C69E27C5C9FFFF0E9EB600
:106B000002D0E82EFCD79E96C69E26C5C9FFFF0E72
:106B10009EB602D0E82EFCD79E96C69E25C5C9FF1C
:106B2000FF0E9EB602D0E82EFCD79E96C69EC95296
:106B3000FF0E9EB602D0E82EFCD7898A0F01C950FD
:106B4000FF0A1DE005012E51130A05E005012E5133
:106B5000170A0BE012000501000E256F000E266FCC
:106B6000100E276F000E286F12000501000E256F12
:106B7000000E266F000E276F010E286F1200050110
:106B8000256B266B276B286B05012E51130A05E038
:106B900005012E51170A0CE012000501000E216FAD
:106BA000000E226F080E236F000E246FE1EF35F008
:106BB0000501000E216F000E226F800E236F000E64
:106BC000246F21C500F122C501F123C502F124C5BE
:106BD00003F125C504F126C505F127C506F128C531
:106BE00007F102EC2FF000C125F501C126F502C125
:106BF00027F503C128F5899A400EC76E200EC66E90
:106C00009E96C69E030EC96EFF0E9EB602D0E82E5B
:106C1000FCD79E96C69E27C5C9FFFF0E9EB602D022
:106C2000E82EFCD79E96C69E26C5C9FFFF0E9EB6CF
:106C300002D0E82EFCD79E96C69E25C5C9FFFF0E42
:106C40009EB602D0E82EFCD79E96C69EC952FF0E75
:106C50009EB602D0E82EFCD7898AC950FF0A08E107
:106C600004C125F505C126F506C127F507C128F59C
:106C7000D890050124332333223321332151F00BE3
:106C8000216F050121674CEF36F022674CEF36F09B
:106C900023674CEF36F02467E1EF35F00501200E55
:106CA0002527E86A2623E86A2723E86A28231200B2
:106CB000E86A05012E51130A06E005012E51170A54
:106CC0000BE0020E120005012851000A03E12751D2
:106CD000F00B07E0010E120005012851000A01E047
:106CE000010E120029C500F12AC501F12BC502F1E0
:106CF0002CC503F125C504F126C505F127C506F10C
:106D000028C507F1B1EC30F003BF120058EC36F0A3
:106D1000D8A4EAEF36F0899A400EC76E200EC66EF0
:106D20009E96C69E060EC96EFF0E9EB602D0E82E37
:106D3000FCD7898A899A9E96C69E020EC96EFF0E5E
:106D40009EB602D0E82EFCD79E96C69E27C5C9FFE8
:106D5000FF0E9EB602D0E82EFCD79E96C69E26C594
:106D6000C9FFFF0E9EB602D0E82EFCD79E96C69EA7
:106D700025C5C9FFFF0E9EB602D0E82EFCD79E9611
:106D8000C69E000EC96EFF0E9EB602D0E82EFCD73E
:106D9000898A899A9E96C69E050EC96EFF0E9EB67A
:106DA00002D0E82EFCD79E96C69EC952FF0E9EB614
:106DB00002D0E82EFCD7C9B0D3EF36F0898A05019E
:106DC000200E2527E86A2623E86A2723E86A282375
:106DD00072EF36F01200899A400EC76E200EC66E12
:106DE0009E96C69E060EC96EFF0E9EB602D0E82E77
:106DF000FCD7898A899A9E96C69EC70EC96EFF0ED9
:106E00009EB602D0E82EFCD7898A0501256B266B39
:106E1000276B286B1200899A400EC76E200EC66E33
:106E20009E96C69E050EC96EFF0E9EB602D0E82E37
:106E3000FCD79E96C69EC952FF0E9EB602D0E82E83
:106E4000FCD7C9CF37F5898A1200899A400EC76EE0
:106E5000200EC66E9E96C69EB90EC96EFF0E9EB6D9
:106E600002D0E82EFCD7898A1200899A400EC76E9C
:106E7000200EC66E9E96C69EAB0EC96EFF0E9EB6C7
:106E800002D0E82EFCD7898AFF0EE82EFED712002A
:106E900058EC36F0D8A41200899A400EC76E200E26
:106EA000C66E9E96C69E030EC96EFF0E9EB602D09B
:106EB000E82EFCD79E96C69E27C5C9FFFF0E9EB63C
:106EC00002D0E82EFCD79E96C69E26C5C9FFFF0EAF
:106ED0009EB602D0E82EFCD79E96C69E25C5C9FF59
:106EE000FF0E9EB602D0E82EFCD79E96C69EC952D3
:106EF000FF0E9EB602D0E82EFCD7898A0F01C9503A
:106F0000FF0AD8A4C7EF38F00501FE0E376F050160
:106F1000FF0E536FFF0E546FFF0E556FFF0E566F2F
:106F200015A63799158677EC32F0AFC538F5B0C5A0
:106F300039F5B1C53AF5B2C53BF5B3C53CF5B4C5B5
:106F40003DF5B5C53EF50784BAC166F1BBC167F131
:106F5000BCC168F1BDC169F14BC14FF14CC150F1E9
:106F60004DC151F14EC152F157C159F158C15AF1B9
:106F700000011650010AD8B4CCEF37F000011650CA
:106F8000020AD8B4F1EF37F000011650040AD8B461
:106F900016EF38F0C7EF38F00501476B486B496BC7
:106FA0004A6B05014B6B4C6B4D6B4E6B05014F6B88
:106FB000506B516B526B8BA0379B97EC22F000C14A
:106FC000DAF101C1DBF102C1DCF103C1DDF100C185
:106FD0003FF501C140F502C141F503C142F535EF6E
:106FE00038F00501476B486B496B4A6B05014B6BE9
:106FF0004C6B4D6B4E6B05014F6B506B516B526B75
:1070000097EC22F000C1DAF101C1DBF102C1DCF141
:1070100003C1DDF194EC23F000C147F501C148F54F
:1070200002C149F503C14AF5C7EF38F0379BDAC111
:107030003FF5DBC140F5DCC141F5DDC142F597EC20
:1070400022F000C14BF501C14CF502C14DF503C161
:107050004EF594EC23F000C14FF501C150F502C18B
:1070600051F503C152F535EF38F00501616740EF86
:1070700038F0626740EF38F0636740EF38F06467DC
:1070800044EF38F059EF38F0DAC100F1DBC101F11B
:10709000DCC102F1DDC103F161C504F162C505F196
:1070A00063C506F164C507F1B1EC30F003BFC7EF6B
:1070B00038F059C143F55AC144F5B9C545F5050144
:1070C000210E326F899A400EC76E200EC66E9E96B4
:1070D000C69E060EC96EFF0E9EB602D0E82EFCD7E5
:1070E000898A899A9E96C69E020EC96EFF0E9EB62A
:1070F00002D0E82EFCD79E96C69E27C5C9FFFF0E7C
:107100009EB602D0E82EFCD79E96C69E26C5C9FF25
:10711000FF0E9EB602D0E82EFCD79E96C69E25C5D1
:10712000C9FFFF0E9EB602D0E82EFCD725EE37F041
:10713000322F02D0A7EF38F09E96C69EDECFC9FF51
:10714000FF0E9EB602D0E82EFCD798EF38F0898A61
:10715000899A9E96C69E050EC96EFF0E9EB602D0F7
:10716000E82EFCD79E96C69EC952FF0E9EB602D050
:10717000E82EFCD7C9B0B2EF38F0898A0501200E9D
:107180002527E86A2623E86A2723E86A282315903A
:107190000794120021C500F122C501F123C502F1B7
:1071A00024C503F1899A400EC76E200EC66E9E96C6
:1071B000C69E0B0EC96EFF0E9EB602D0E82EFCD7FF
:1071C0009E96C69E02C1C9FFFF0E9EB602D0E82E53
:1071D000FCD79E96C69E01C1C9FFFF0E9EB602D087
:1071E000E82EFCD79E96C69E00C1C9FFFF0E9EB634
:1071F00002D0E82EFCD79E96C69EC952FF0E9EB6C0
:1072000002D0E82EFCD725EE37F00501200E326FB4
:107210009E96C69EC952FF0E9EB602D0E82EFCD79F
:10722000C9CFDEFF322F08EF39F0898A1200899A20
:10723000400EC76E200EC66E9E96C69E900EC96EFC
:10724000FF0E9EB602D0E82EFCD79E96C69E000E7C
:10725000C96EFF0E9EB602D0E82EFCD79E96C69E43
:10726000000EC96EFF0E9EB602D0E82EFCD79E9689
:10727000C69E000EC96EFF0E9EB602D0E82EFCD749
:107280009E96C69EC952FF0E9EB602D0E82EFCD72F
:10729000C9CF2DF59E96C69EC952FF0E9EB602D04E
:1072A000E82EFCD7C9CF2EF5898A120077EC32F090
:1072B00005012F51010A61E005012F51020A16E074
:1072C00005012F51030A1BE005012F51040A26E096
:1072D00005012F51050A2DE005012F51060A3BE05B
:1072E00005012F51070A41E0BDEF39F015B012003A
:1072F000602FBBEF39F05FC560F5BDEF39F0B0C569
:1073000000F101010F0E001701010051000A35E0E4
:1073100001010051050A31E0BBEF39F0B0C500F1C1
:1073200001010F0E001701010051000A26E0BBEF1A
:1073300039F00501B051000A20E00501B051150AED
:107340001CE00501B051300A18E00501B051450AB2
:1073500014E0BBEF39F00501B051000A0EE0050161
:10736000B051300A0AE0BBEF39F00501B051000A14
:1073700004E0BBEF39F015901200158012008B90DD
:107380007DEC2FF0B9C5E8FFD70802E37DEC2FF0C4
:10739000B9C5E8FFC80802E37DEC2FF0B9C5E8FFE6
:1073A000B90802E37DEC2FF0B9C5E8FFAA0802E3B3
:1073B0007DEC2FF0B9C5E8FF9B0802E37DEC2FF0D0
:1073C00025EC37F0F29CF29E8B94C69AC290948280
:1073D000948C720ED36ED3A4FED789968A90939024
:1073E000F29AF2949D909E909D929E92F298F292C3
:1073F000E7EC33F0FF0EE8CF00F0E82EFED7002ECA
:10740000FCD7F290F2868150FF0EE82EFED7F29064
:1074100081A80DEF3AF0F29E0300700ED36EF29643
:0E742000F290158403809EEC2FF09AEF0BF093
:10BF0000E844F926000C160C2B0C3F0C520C640C68
:10BF1000760C860C960CA50CB30CC10CCF0CDC0C6B
:06BF2000E80CF40C000C1B
:0200000400F00A
:0100C800FD3A
:00000001FF
